Component: ARM Compiler 5.06 update 6 (build 750) Tool: armlink [4d35ed]

==============================================================================

Small function inlining results

Inlined total of 0 calls.

==============================================================================

Section Cross References

    system_nuc200series.o(i.SystemCoreClockUpdate) refers to uidiv.o(.text) for __aeabi_uidivmod
    system_nuc200series.o(i.SystemCoreClockUpdate) refers to system_nuc200series.o(.data) for .data
    startup_nuc200series.o(RESET) refers to startup_nuc200series.o(STACK) for __initial_sp
    startup_nuc200series.o(RESET) refers to startup_nuc200series.o(.text) for Reset_Handler
    startup_nuc200series.o(RESET) refers to retarget.o(.emb_text) for HardFault_Handler
    startup_nuc200series.o(RESET) refers to chip_uip_interrupt.o(i.BOD_IRQHandler) for BOD_IRQHandler
    startup_nuc200series.o(RESET) refers to chip_uip_interrupt.o(i.WDT_IRQHandler) for WDT_IRQHandler
    startup_nuc200series.o(RESET) refers to chip_uip_interrupt.o(i.EINT0_IRQHandler) for EINT0_IRQHandler
    startup_nuc200series.o(RESET) refers to chip_uip_interrupt.o(i.EINT1_IRQHandler) for EINT1_IRQHandler
    startup_nuc200series.o(RESET) refers to chip_uip_interrupt.o(i.GPAB_IRQHandler) for GPAB_IRQHandler
    startup_nuc200series.o(RESET) refers to chip_uip_interrupt.o(i.GPCDEF_IRQHandler) for GPCDEF_IRQHandler
    startup_nuc200series.o(RESET) refers to chip_uip_interrupt.o(i.PWMA_IRQHandler) for PWMA_IRQHandler
    startup_nuc200series.o(RESET) refers to chip_uip_interrupt.o(i.PWMB_IRQHandler) for PWMB_IRQHandler
    startup_nuc200series.o(RESET) refers to chip_uip_interrupt.o(i.TMR0_IRQHandler) for TMR0_IRQHandler
    startup_nuc200series.o(RESET) refers to chip_uip_interrupt.o(i.TMR1_IRQHandler) for TMR1_IRQHandler
    startup_nuc200series.o(RESET) refers to chip_uip_interrupt.o(i.TMR2_IRQHandler) for TMR2_IRQHandler
    startup_nuc200series.o(RESET) refers to chip_uip_interrupt.o(i.TMR3_IRQHandler) for TMR3_IRQHandler
    startup_nuc200series.o(RESET) refers to chip_uip_interrupt.o(i.UART02_IRQHandler) for UART02_IRQHandler
    startup_nuc200series.o(RESET) refers to chip_uip_interrupt.o(i.UART1_IRQHandler) for UART1_IRQHandler
    startup_nuc200series.o(RESET) refers to chip_uip_interrupt.o(i.SPI0_IRQHandler) for SPI0_IRQHandler
    startup_nuc200series.o(RESET) refers to chip_uip_interrupt.o(i.SPI1_IRQHandler) for SPI1_IRQHandler
    startup_nuc200series.o(RESET) refers to chip_uip_interrupt.o(i.SPI2_IRQHandler) for SPI2_IRQHandler
    startup_nuc200series.o(RESET) refers to chip_uip_interrupt.o(i.SPI3_IRQHandler) for SPI3_IRQHandler
    startup_nuc200series.o(RESET) refers to chip_uip_interrupt.o(i.I2C0_IRQHandler) for I2C0_IRQHandler
    startup_nuc200series.o(RESET) refers to chip_uip_interrupt.o(i.I2C1_IRQHandler) for I2C1_IRQHandler
    startup_nuc200series.o(RESET) refers to chip_uip_interrupt.o(i.CAN0_IRQHandler) for CAN0_IRQHandler
    startup_nuc200series.o(RESET) refers to chip_uip_interrupt.o(i.CAN1_IRQHandler) for CAN1_IRQHandler
    startup_nuc200series.o(RESET) refers to chip_uip_interrupt.o(i.SC012_IRQHandler) for SC012_IRQHandler
    startup_nuc200series.o(RESET) refers to chip_uip_interrupt.o(i.USBD_IRQHandler) for USBD_IRQHandler
    startup_nuc200series.o(RESET) refers to chip_uip_interrupt.o(i.PS2_IRQHandler) for PS2_IRQHandler
    startup_nuc200series.o(RESET) refers to chip_uip_interrupt.o(i.ACMP_IRQHandler) for ACMP_IRQHandler
    startup_nuc200series.o(RESET) refers to chip_uip_interrupt.o(i.PDMA_IRQHandler) for PDMA_IRQHandler
    startup_nuc200series.o(RESET) refers to chip_uip_interrupt.o(i.I2S_IRQHandler) for I2S_IRQHandler
    startup_nuc200series.o(RESET) refers to chip_uip_interrupt.o(i.PWRWU_IRQHandler) for PWRWU_IRQHandler
    startup_nuc200series.o(RESET) refers to chip_uip_interrupt.o(i.ADC_IRQHandler) for ADC_IRQHandler
    startup_nuc200series.o(RESET) refers to chip_uip_interrupt.o(i.RTC_IRQHandler) for RTC_IRQHandler
    startup_nuc200series.o(.text) refers to system_nuc200series.o(i.SystemInit) for SystemInit
    startup_nuc200series.o(.text) refers to entry.o(.ARM.Collect$$$$00000000) for __main
    app_cfg.o(.data) refers to app_cfg.o(.data) for AppAlarmBase
    app_cfg.o(.data) refers to app_cfg.o(.data) for AppCounter
    app_cfg.o(.data) refers to app_cfg.o(.data) for AppMsgBuf
    app_cfg.o(.data) refers to demo.o(i.TASK_0) for TASK_0
    app_cfg.o(.data) refers to app_cfg.o(.bss) for Task_0_Stack
    app_cfg.o(.data) refers to demo.o(i.TASK_1) for TASK_1
    app_cfg.o(.data) refers to app_cfg.o(.bss) for Task_1_Stack
    app_cfg.o(.data) refers to demo.o(i.TASK_2) for TASK_2
    app_cfg.o(.data) refers to app_cfg.o(.bss) for Task_2_Stack
    app_cfg.o(.data) refers to demo.o(i.TASK_3) for TASK_3
    app_cfg.o(.data) refers to app_cfg.o(.bss) for Task_3_Stack
    app_cfg.o(.data) refers to demo.o(i.TASK_4) for TASK_4
    app_cfg.o(.data) refers to app_cfg.o(.bss) for Task_4_Stack
    app_cfg.o(.data) refers to demo.o(i.AppIdleTask) for AppIdleTask
    app_cfg.o(.data) refers to app_cfg.o(.bss) for Task_App_Idle_Stack
    app_int_cfg.o(.data) refers to app_int_cfg.o(i.Chip_NUC200_ADC_ISR_Handler_Callback) for Chip_NUC200_ADC_ISR_Handler_Callback
    app_int_cfg.o(.data) refers to init.o(i.ADC_IRQHandler_Process) for ADC_IRQHandler_Process
    app_int_cfg.o(.data) refers to app_int_cfg.o(.data) for ChipNUC200ADCIntHandlingData
    demo.o(i.TASK_0) refers to init.o(i.UART0_Init) for UART0_Init
    demo.o(i.TASK_0) refers to uip_kernel_event.o(i.UIP_WaitEvent) for UIP_WaitEvent
    demo.o(i.TASK_0) refers to uip_kernel_event.o(i.UIP_ClearEvent) for UIP_ClearEvent
    demo.o(i.TASK_1) refers to uip_kernel_event.o(i.UIP_WaitEvent) for UIP_WaitEvent
    demo.o(i.TASK_1) refers to uip_kernel_event.o(i.UIP_ClearEvent) for UIP_ClearEvent
    demo.o(i.TASK_2) refers to uip_kernel_resource.o(i.UIP_GetResource) for UIP_GetResource
    demo.o(i.TASK_2) refers to init.o(i.GetAVDDVoltage) for GetAVDDVoltage
    demo.o(i.TASK_2) refers to printf5.o(i.__0sprintf$5) for __2sprintf
    demo.o(i.TASK_2) refers to uip_kernel_message.o(i.UIP_SendMessage) for UIP_SendMessage
    demo.o(i.TASK_2) refers to uip_kernel_resource.o(i.UIP_ReleaseResource) for UIP_ReleaseResource
    demo.o(i.TASK_3) refers to uip_kernel_resource.o(i.UIP_GetResource) for UIP_GetResource
    demo.o(i.TASK_3) refers to adc.o(i.ADC_DisableInt) for ADC_DisableInt
    demo.o(i.TASK_3) refers to uip_kernel_resource.o(i.UIP_ReleaseResource) for UIP_ReleaseResource
    demo.o(i.TASK_4) refers to uip_kernel_message.o(i.UIP_ReceiveMessage) for UIP_ReceiveMessage
    demo.o(i.TASK_4) refers to atoi.o(.text) for atoi
    demo.o(i.TASK_4) refers to printf5.o(i.__0printf$5) for __2printf
    demo.o(i.TASK_4) refers to uip_kernel_task.o(i.UIP_TerminateTask) for UIP_TerminateTask
    demo.o(i.main) refers to hardware_init.o(i.Hardware_Init) for Hardware_Init
    demo.o(i.main) refers to init.o(i.pre_main_init) for pre_main_init
    demo.o(i.main) refers to uip_kernel_common.o(i.StartOS) for StartOS
    demo.o(i.main) refers to uip_kernel_common.o(.data) for uipIdleTaskID
    demo.o(i.uipAppInitialize) refers to uip_kernel_common.o(i.uipTaskInitialize) for uipTaskInitialize
    demo.o(i.uipAppInitialize) refers to uip_kernel_common.o(i.uipAlarmInitialize) for uipAlarmInitialize
    demo.o(i.uipAppInitialize) refers to uip_kernel_common.o(i.uipResInitialize) for uipResInitialize
    demo.o(i.uipAppInitialize) refers to uip_kernel_common.o(i.uipMsgInitialize) for uipMsgInitialize
    demo.o(i.uipAppInitialize) refers to hardware_init.o(i.Kernel_System_Tick_Init) for Kernel_System_Tick_Init
    demo.o(i.uipAppInitialize) refers to app_cfg.o(.data) for AppTaskNumber
    demo.o(i.uipAppInitialize) refers to app_cfg.o(.data) for AppTask
    demo.o(i.uipAppInitialize) refers to app_cfg.o(.data) for AppAlarmNumber
    demo.o(i.uipAppInitialize) refers to app_cfg.o(.data) for AppAlarm
    demo.o(i.uipAppInitialize) refers to app_cfg.o(.data) for AppResNumber
    demo.o(i.uipAppInitialize) refers to app_cfg.o(.data) for AppRes
    demo.o(i.uipAppInitialize) refers to app_cfg.o(.data) for AppMsgNumber
    demo.o(i.uipAppInitialize) refers to app_cfg.o(.data) for AppMsg
    init.o(i.ADC_IRQHandler_Process) refers to uip_kernel_event.o(i.UIP_SetEvent) for UIP_SetEvent
    init.o(i.GetAVDDCodeByADC) refers to adc.o(i.ADC_Open) for ADC_Open
    init.o(i.GetAVDDCodeByADC) refers to adc.o(i.ADC_EnableInt) for ADC_EnableInt
    init.o(i.GetAVDDCodeByADC) refers to uip_kernel_event.o(i.UIP_WaitEvent) for UIP_WaitEvent
    init.o(i.GetAVDDCodeByADC) refers to uip_kernel_event.o(i.UIP_ClearEvent) for UIP_ClearEvent
    init.o(i.GetAVDDCodeByADC) refers to system_nuc200series.o(.data) for CyclesPerUs
    init.o(i.GetAVDDVoltage) refers to init.o(i.GetAVDDCodeByADC) for GetAVDDCodeByADC
    init.o(i.GetAVDDVoltage) refers to uldiv.o(.text) for __aeabi_uldivmod
    init.o(i.SYS_Init) refers to clk.o(i.CLK_EnableXtalRC) for CLK_EnableXtalRC
    init.o(i.SYS_Init) refers to clk.o(i.CLK_WaitClockReady) for CLK_WaitClockReady
    init.o(i.SYS_Init) refers to clk.o(i.CLK_SetHCLK) for CLK_SetHCLK
    init.o(i.SYS_Init) refers to clk.o(i.CLK_SetCoreClock) for CLK_SetCoreClock
    init.o(i.SYS_Init) refers to clk.o(i.CLK_EnableModuleClock) for CLK_EnableModuleClock
    init.o(i.SYS_Init) refers to clk.o(i.CLK_SetModuleClock) for CLK_SetModuleClock
    init.o(i.UART0_Init) refers to sys.o(i.SYS_ResetModule) for SYS_ResetModule
    init.o(i.UART0_Init) refers to uart.o(i.UART_Open) for UART_Open
    init.o(i.pre_main_init) refers to init.o(i.SYS_Init) for SYS_Init
    retarget.o(.emb_text) refers to retarget.o(i.Hard_Fault_Handler) for Hard_Fault_Handler
    retarget.o(i.Hard_Fault_Handler) refers to printf5.o(i.__0printf$5) for __2printf
    retarget.o(i.Hard_Fault_Handler) refers to retarget.o(i.stackDump) for stackDump
    retarget.o(i.SendChar) refers to retarget.o(i.SendChar_ToUART) for SendChar_ToUART
    retarget.o(i._ttywrch) refers to retarget.o(i.SendChar_ToUART) for SendChar_ToUART
    retarget.o(i.fgetc) refers to retarget.o(i.GetChar) for GetChar
    retarget.o(i.fputc) refers to retarget.o(i.SendChar_ToUART) for SendChar_ToUART
    retarget.o(i.stackDump) refers to printf5.o(i.__0printf$5) for __2printf
    clk.o(i.CLK_DisableCKO) refers to clk.o(i.CLK_DisableModuleClock) for CLK_DisableModuleClock
    clk.o(i.CLK_DisableModuleClock) refers to clk.o(.constdata) for .constdata
    clk.o(i.CLK_EnableCKO) refers to clk.o(i.CLK_EnableModuleClock) for CLK_EnableModuleClock
    clk.o(i.CLK_EnableCKO) refers to clk.o(i.CLK_SetModuleClock) for CLK_SetModuleClock
    clk.o(i.CLK_EnableModuleClock) refers to clk.o(.constdata) for .constdata
    clk.o(i.CLK_EnablePLL) refers to clk.o(i.CLK_WaitClockReady) for CLK_WaitClockReady
    clk.o(i.CLK_EnablePLL) refers to uidiv.o(.text) for __aeabi_uidivmod
    clk.o(i.CLK_GetCPUFreq) refers to system_nuc200series.o(i.SystemCoreClockUpdate) for SystemCoreClockUpdate
    clk.o(i.CLK_GetCPUFreq) refers to system_nuc200series.o(.data) for SystemCoreClock
    clk.o(i.CLK_GetHCLKFreq) refers to system_nuc200series.o(i.SystemCoreClockUpdate) for SystemCoreClockUpdate
    clk.o(i.CLK_GetHCLKFreq) refers to system_nuc200series.o(.data) for SystemCoreClock
    clk.o(i.CLK_GetPCLKFreq) refers to system_nuc200series.o(i.SystemCoreClockUpdate) for SystemCoreClockUpdate
    clk.o(i.CLK_GetPCLKFreq) refers to system_nuc200series.o(.data) for SystemCoreClock
    clk.o(i.CLK_SetCoreClock) refers to clk.o(i.CLK_EnablePLL) for CLK_EnablePLL
    clk.o(i.CLK_SetCoreClock) refers to clk.o(i.CLK_SetHCLK) for CLK_SetHCLK
    clk.o(i.CLK_SetHCLK) refers to system_nuc200series.o(i.SystemCoreClockUpdate) for SystemCoreClockUpdate
    clk.o(i.CLK_SetModuleClock) refers to clk.o(.constdata) for .constdata
    uart.o(i.CLK_GetPLLClockFreq) refers to uidiv.o(.text) for __aeabi_uidivmod
    uart.o(i.UART_Open) refers to uart.o(i.CLK_GetPLLClockFreq) for CLK_GetPLLClockFreq
    uart.o(i.UART_Open) refers to uidiv.o(.text) for __aeabi_uidivmod
    uart.o(i.UART_Open) refers to uart.o(.constdata) for .constdata
    uart.o(i.UART_SelectIrDAMode) refers to uart.o(i.CLK_GetPLLClockFreq) for CLK_GetPLLClockFreq
    uart.o(i.UART_SelectIrDAMode) refers to uidiv.o(.text) for __aeabi_uidivmod
    uart.o(i.UART_SelectIrDAMode) refers to uart.o(.constdata) for .constdata
    uart.o(i.UART_SetLine_Config) refers to uart.o(i.CLK_GetPLLClockFreq) for CLK_GetPLLClockFreq
    uart.o(i.UART_SetLine_Config) refers to uidiv.o(.text) for __aeabi_uidivmod
    uart.o(i.UART_SetLine_Config) refers to uart.o(.constdata) for .constdata
    chip_uip_interrupt.o(i.ACMP_IRQHandler) refers to uip_kernel_isr_engine.o(i.uipInterruptServiceEngine) for uipInterruptServiceEngine
    chip_uip_interrupt.o(i.ACMP_IRQHandler) refers to uip_kernel_common.o(.data) for uipIntTableID
    chip_uip_interrupt.o(i.ADC_IRQHandler) refers to uip_kernel_isr_engine.o(i.uipInterruptServiceEngine) for uipInterruptServiceEngine
    chip_uip_interrupt.o(i.ADC_IRQHandler) refers to uip_kernel_common.o(.data) for uipIntTableID
    chip_uip_interrupt.o(i.BOD_IRQHandler) refers to uip_kernel_isr_engine.o(i.uipInterruptServiceEngine) for uipInterruptServiceEngine
    chip_uip_interrupt.o(i.BOD_IRQHandler) refers to uip_kernel_common.o(.data) for uipIntTableID
    chip_uip_interrupt.o(i.CAN0_IRQHandler) refers to uip_kernel_isr_engine.o(i.uipInterruptServiceEngine) for uipInterruptServiceEngine
    chip_uip_interrupt.o(i.CAN0_IRQHandler) refers to uip_kernel_common.o(.data) for uipIntTableID
    chip_uip_interrupt.o(i.CAN1_IRQHandler) refers to uip_kernel_isr_engine.o(i.uipInterruptServiceEngine) for uipInterruptServiceEngine
    chip_uip_interrupt.o(i.CAN1_IRQHandler) refers to uip_kernel_common.o(.data) for uipIntTableID
    chip_uip_interrupt.o(i.Chip_UIP_InterruptInit) refers to chip_uip_interrupt.o(i.Chip_UIP_InterruptRegisterHandler) for Chip_UIP_InterruptRegisterHandler
    chip_uip_interrupt.o(i.Chip_UIP_InterruptInit) refers to app_int_cfg.o(.data) for UIP_Exc_VectorTable
    chip_uip_interrupt.o(i.Chip_UIP_InterruptInit) refers to chip_uip_interrupt.o(i.Chip_UIP_InterruptNullHandler) for Chip_UIP_InterruptNullHandler
    chip_uip_interrupt.o(i.Chip_UIP_InterruptRegisterHandler) refers to app_int_cfg.o(.data) for UIP_Exc_VectorTable
    chip_uip_interrupt.o(i.Chip_UIP_InterruptRemoveHandler) refers to chip_uip_interrupt.o(i.Chip_UIP_InterruptRegisterHandler) for Chip_UIP_InterruptRegisterHandler
    chip_uip_interrupt.o(i.Chip_UIP_InterruptRemoveHandler) refers to chip_uip_interrupt.o(i.Chip_UIP_InterruptNullHandler) for Chip_UIP_InterruptNullHandler
    chip_uip_interrupt.o(i.Chip_UIP_Kernel_Tick_ISR_Handler) refers to uip_kernel_time.o(i.uipSystemCounterHandler) for uipSystemCounterHandler
    chip_uip_interrupt.o(i.EINT0_IRQHandler) refers to uip_kernel_isr_engine.o(i.uipInterruptServiceEngine) for uipInterruptServiceEngine
    chip_uip_interrupt.o(i.EINT0_IRQHandler) refers to uip_kernel_common.o(.data) for uipIntTableID
    chip_uip_interrupt.o(i.EINT1_IRQHandler) refers to uip_kernel_isr_engine.o(i.uipInterruptServiceEngine) for uipInterruptServiceEngine
    chip_uip_interrupt.o(i.EINT1_IRQHandler) refers to uip_kernel_common.o(.data) for uipIntTableID
    chip_uip_interrupt.o(i.GPAB_IRQHandler) refers to uip_kernel_isr_engine.o(i.uipInterruptServiceEngine) for uipInterruptServiceEngine
    chip_uip_interrupt.o(i.GPAB_IRQHandler) refers to uip_kernel_common.o(.data) for uipIntTableID
    chip_uip_interrupt.o(i.GPCDEF_IRQHandler) refers to uip_kernel_isr_engine.o(i.uipInterruptServiceEngine) for uipInterruptServiceEngine
    chip_uip_interrupt.o(i.GPCDEF_IRQHandler) refers to uip_kernel_common.o(.data) for uipIntTableID
    chip_uip_interrupt.o(i.I2C0_IRQHandler) refers to uip_kernel_isr_engine.o(i.uipInterruptServiceEngine) for uipInterruptServiceEngine
    chip_uip_interrupt.o(i.I2C0_IRQHandler) refers to uip_kernel_common.o(.data) for uipIntTableID
    chip_uip_interrupt.o(i.I2C1_IRQHandler) refers to uip_kernel_isr_engine.o(i.uipInterruptServiceEngine) for uipInterruptServiceEngine
    chip_uip_interrupt.o(i.I2C1_IRQHandler) refers to uip_kernel_common.o(.data) for uipIntTableID
    chip_uip_interrupt.o(i.I2S_IRQHandler) refers to uip_kernel_isr_engine.o(i.uipInterruptServiceEngine) for uipInterruptServiceEngine
    chip_uip_interrupt.o(i.I2S_IRQHandler) refers to uip_kernel_common.o(.data) for uipIntTableID
    chip_uip_interrupt.o(i.InterruptHandler) refers to uip_kernel_common.o(.data) for uipIntTableID
    chip_uip_interrupt.o(i.InterruptHandler) refers to app_int_cfg.o(.data) for UIP_Exc_VectorTable
    chip_uip_interrupt.o(i.InterruptHandler) refers to app_int_cfg.o(.data) for AppIntNumber
    chip_uip_interrupt.o(i.PDMA_IRQHandler) refers to uip_kernel_isr_engine.o(i.uipInterruptServiceEngine) for uipInterruptServiceEngine
    chip_uip_interrupt.o(i.PDMA_IRQHandler) refers to uip_kernel_common.o(.data) for uipIntTableID
    chip_uip_interrupt.o(i.PS2_IRQHandler) refers to uip_kernel_isr_engine.o(i.uipInterruptServiceEngine) for uipInterruptServiceEngine
    chip_uip_interrupt.o(i.PS2_IRQHandler) refers to uip_kernel_common.o(.data) for uipIntTableID
    chip_uip_interrupt.o(i.PWMA_IRQHandler) refers to uip_kernel_isr_engine.o(i.uipInterruptServiceEngine) for uipInterruptServiceEngine
    chip_uip_interrupt.o(i.PWMA_IRQHandler) refers to uip_kernel_common.o(.data) for uipIntTableID
    chip_uip_interrupt.o(i.PWMB_IRQHandler) refers to uip_kernel_isr_engine.o(i.uipInterruptServiceEngine) for uipInterruptServiceEngine
    chip_uip_interrupt.o(i.PWMB_IRQHandler) refers to uip_kernel_common.o(.data) for uipIntTableID
    chip_uip_interrupt.o(i.PWRWU_IRQHandler) refers to uip_kernel_isr_engine.o(i.uipInterruptServiceEngine) for uipInterruptServiceEngine
    chip_uip_interrupt.o(i.PWRWU_IRQHandler) refers to uip_kernel_common.o(.data) for uipIntTableID
    chip_uip_interrupt.o(i.RTC_IRQHandler) refers to uip_kernel_isr_engine.o(i.uipInterruptServiceEngine) for uipInterruptServiceEngine
    chip_uip_interrupt.o(i.RTC_IRQHandler) refers to uip_kernel_common.o(.data) for uipIntTableID
    chip_uip_interrupt.o(i.SC012_IRQHandler) refers to uip_kernel_isr_engine.o(i.uipInterruptServiceEngine) for uipInterruptServiceEngine
    chip_uip_interrupt.o(i.SC012_IRQHandler) refers to uip_kernel_common.o(.data) for uipIntTableID
    chip_uip_interrupt.o(i.SPI0_IRQHandler) refers to uip_kernel_isr_engine.o(i.uipInterruptServiceEngine) for uipInterruptServiceEngine
    chip_uip_interrupt.o(i.SPI0_IRQHandler) refers to uip_kernel_common.o(.data) for uipIntTableID
    chip_uip_interrupt.o(i.SPI1_IRQHandler) refers to uip_kernel_isr_engine.o(i.uipInterruptServiceEngine) for uipInterruptServiceEngine
    chip_uip_interrupt.o(i.SPI1_IRQHandler) refers to uip_kernel_common.o(.data) for uipIntTableID
    chip_uip_interrupt.o(i.SPI2_IRQHandler) refers to uip_kernel_isr_engine.o(i.uipInterruptServiceEngine) for uipInterruptServiceEngine
    chip_uip_interrupt.o(i.SPI2_IRQHandler) refers to uip_kernel_common.o(.data) for uipIntTableID
    chip_uip_interrupt.o(i.SPI3_IRQHandler) refers to uip_kernel_isr_engine.o(i.uipInterruptServiceEngine) for uipInterruptServiceEngine
    chip_uip_interrupt.o(i.SPI3_IRQHandler) refers to uip_kernel_common.o(.data) for uipIntTableID
    chip_uip_interrupt.o(i.TMR0_IRQHandler) refers to uip_kernel_isr_engine.o(i.uipInterruptServiceEngine) for uipInterruptServiceEngine
    chip_uip_interrupt.o(i.TMR0_IRQHandler) refers to uip_kernel_common.o(.data) for uipIntTableID
    chip_uip_interrupt.o(i.TMR1_IRQHandler) refers to uip_kernel_isr_engine.o(i.uipInterruptServiceEngine) for uipInterruptServiceEngine
    chip_uip_interrupt.o(i.TMR1_IRQHandler) refers to uip_kernel_common.o(.data) for uipIntTableID
    chip_uip_interrupt.o(i.TMR2_IRQHandler) refers to uip_kernel_isr_engine.o(i.uipInterruptServiceEngine) for uipInterruptServiceEngine
    chip_uip_interrupt.o(i.TMR2_IRQHandler) refers to uip_kernel_common.o(.data) for uipIntTableID
    chip_uip_interrupt.o(i.TMR3_IRQHandler) refers to uip_kernel_isr_engine.o(i.uipInterruptServiceEngine) for uipInterruptServiceEngine
    chip_uip_interrupt.o(i.TMR3_IRQHandler) refers to uip_kernel_common.o(.data) for uipIntTableID
    chip_uip_interrupt.o(i.UART02_IRQHandler) refers to uip_kernel_isr_engine.o(i.uipInterruptServiceEngine) for uipInterruptServiceEngine
    chip_uip_interrupt.o(i.UART02_IRQHandler) refers to uip_kernel_common.o(.data) for uipIntTableID
    chip_uip_interrupt.o(i.UART1_IRQHandler) refers to uip_kernel_isr_engine.o(i.uipInterruptServiceEngine) for uipInterruptServiceEngine
    chip_uip_interrupt.o(i.UART1_IRQHandler) refers to uip_kernel_common.o(.data) for uipIntTableID
    chip_uip_interrupt.o(i.USBD_IRQHandler) refers to uip_kernel_isr_engine.o(i.uipInterruptServiceEngine) for uipInterruptServiceEngine
    chip_uip_interrupt.o(i.USBD_IRQHandler) refers to uip_kernel_common.o(.data) for uipIntTableID
    chip_uip_interrupt.o(i.WDT_IRQHandler) refers to uip_kernel_isr_engine.o(i.uipInterruptServiceEngine) for uipInterruptServiceEngine
    chip_uip_interrupt.o(i.WDT_IRQHandler) refers to uip_kernel_common.o(.data) for uipIntTableID
    chip_uip_interrupt.o(i.uipInterruptHandlingCallback) refers to chip_uip_interrupt.o(i.InterruptHandler) for InterruptHandler
    chip_uip_interrupt.o(i.uipInterruptHandlingCallback) refers to uip_kernel_common.o(.data) for uipLowPowerMode
    hardware_init.o(i.Kernel_System_Tick_Init) refers to uidiv.o(.text) for __aeabi_uidivmod
    hardware_init.o(i.Kernel_System_Tick_Init) refers to system_nuc200series.o(.data) for SystemCoreClock
    uip_kernel_common.o(i.StartOS) refers to uip_kernel_isr_cm.o(CODE) for uipDisableAllInterrupts
    uip_kernel_common.o(i.StartOS) refers to uip_kernel_common.o(i.uipKernelInitialize) for uipKernelInitialize
    uip_kernel_common.o(i.StartOS) refers to demo.o(i.uipAppInitialize) for uipAppInitialize
    uip_kernel_common.o(i.StartOS) refers to uip_kernel_scheduler.o(.data) for uipSystemMode
    uip_kernel_common.o(i.uipAlarmInfoInit) refers to uip_kernel_common.o(.data) for .data
    uip_kernel_common.o(i.uipAlarmInitialize) refers to uip_kernel_common.o(.data) for .data
    uip_kernel_common.o(i.uipKernelInitialize) refers to uip_kernel_common.o(.data) for .data
    uip_kernel_common.o(i.uipKernelInitialize) refers to uip_kernel_common.o(.bss) for .bss
    uip_kernel_common.o(i.uipKernelInitialize) refers to uip_kernel_scheduler.o(.data) for uipPrioGrpArray
    uip_kernel_common.o(i.uipKernelInitialize) refers to uip_kernel_scheduler.o(.data) for uipSchedulerLock
    uip_kernel_common.o(i.uipKernelInitialize) refers to uip_kernel_scheduler.o(.data) for uipNestedInterrupts
    uip_kernel_common.o(i.uipKernelInitialize) refers to uip_kernel_scheduler.o(.data) for uipSystemMode
    uip_kernel_common.o(i.uipKernelInitialize) refers to uip_kernel_scheduler.o(.data) for uipSystemStackPtr
    uip_kernel_common.o(i.uipMsgInfoInit) refers to uip_kernel_common.o(.data) for .data
    uip_kernel_common.o(i.uipMsgInitialize) refers to uip_kernel_common.o(.data) for .data
    uip_kernel_common.o(i.uipResInfoInit) refers to uip_kernel_common.o(.data) for .data
    uip_kernel_common.o(i.uipResInitialize) refers to uip_kernel_common.o(.data) for .data
    uip_kernel_common.o(i.uipTaskInfoInit) refers to uip_kernel_common.o(.data) for .data
    uip_kernel_common.o(i.uipTaskInitialize) refers to uip_kernel_common.o(i.uipTaskStackInit) for uipTaskStackInit
    uip_kernel_common.o(i.uipTaskInitialize) refers to uip_kernel_common.o(.data) for .data
    uip_kernel_common.o(i.uipTaskInitialize) refers to uip_kernel_common.o(.bss) for .bss
    uip_kernel_common.o(i.uipTaskInitialize) refers to uip_kernel_scheduler.o(.data) for uipPrioGroup
    uip_kernel_event.o(i.UIP_ClearEvent) refers to uip_kernel_isr_cm.o(CODE) for uipDisableAllInterrupts
    uip_kernel_event.o(i.UIP_ClearEvent) refers to uip_kernel_scheduler.o(.data) for uipNestedInterrupts
    uip_kernel_event.o(i.UIP_ClearEvent) refers to uip_kernel_scheduler.o(.data) for uipSchedulerLock
    uip_kernel_event.o(i.UIP_ClearEvent) refers to uip_kernel_scheduler.o(.data) for uipCurrentTaskTCBPtr
    uip_kernel_event.o(i.UIP_GetEvent) refers to uip_kernel_isr_cm.o(CODE) for uipDisableAllInterrupts
    uip_kernel_event.o(i.UIP_GetEvent) refers to uip_kernel_scheduler.o(.data) for uipSchedulerLock
    uip_kernel_event.o(i.UIP_GetEvent) refers to uip_kernel_common.o(.data) for uipTCBArray
    uip_kernel_event.o(i.UIP_SetEvent) refers to uip_kernel_isr_cm.o(CODE) for uipDisableAllInterrupts
    uip_kernel_event.o(i.UIP_SetEvent) refers to uip_kernel_scheduler.o(i.uipGetNextPriority) for uipGetNextPriority
    uip_kernel_event.o(i.UIP_SetEvent) refers to uip_kernel_common.o(.data) for uipTCBArray
    uip_kernel_event.o(i.UIP_SetEvent) refers to uip_kernel_scheduler.o(.data) for uipPrioGroup
    uip_kernel_event.o(i.UIP_SetEvent) refers to uip_kernel_scheduler.o(.data) for uipNestedInterrupts
    uip_kernel_event.o(i.UIP_SetEvent) refers to uip_kernel_scheduler.o(.data) for uipSchedulerLock
    uip_kernel_event.o(i.UIP_SetEvent) refers to uip_kernel_common.o(.bss) for uipPriorityToTaskID
    uip_kernel_event.o(i.UIP_WaitEvent) refers to uip_kernel_isr_cm.o(CODE) for uipDisableAllInterrupts
    uip_kernel_event.o(i.UIP_WaitEvent) refers to uip_kernel_scheduler.o(i.uipClearPrioGrpAndArrayBit) for uipClearPrioGrpAndArrayBit
    uip_kernel_event.o(i.UIP_WaitEvent) refers to uip_kernel_scheduler.o(i.uipGetNextTask) for uipGetNextTask
    uip_kernel_event.o(i.UIP_WaitEvent) refers to uip_kernel_scheduler.o(.data) for uipNestedInterrupts
    uip_kernel_event.o(i.UIP_WaitEvent) refers to uip_kernel_scheduler.o(.data) for uipSchedulerLock
    uip_kernel_event.o(i.UIP_WaitEvent) refers to uip_kernel_scheduler.o(.data) for uipCurrentTaskTCBPtr
    uip_kernel_isr_cm.o(CODE) refers to uip_kernel_scheduler.o(i.uipPreContexSwitch) for uipPreContexSwitch
    uip_kernel_isr_cm.o(CODE) refers to uip_kernel_scheduler.o(.data) for uipCurrentTaskTCBPtr
    uip_kernel_isr_engine.o(i.uipInterruptServiceEngine) refers to uip_kernel_isr_cm.o(CODE) for uipDisableAllInterrupts
    uip_kernel_isr_engine.o(i.uipInterruptServiceEngine) refers to chip_uip_interrupt.o(i.uipInterruptHandlingCallback) for uipInterruptHandlingCallback
    uip_kernel_isr_engine.o(i.uipInterruptServiceEngine) refers to uip_kernel_scheduler.o(i.uipGetNextTask) for uipGetNextTask
    uip_kernel_isr_engine.o(i.uipInterruptServiceEngine) refers to uip_kernel_scheduler.o(.data) for uipSystemMode
    uip_kernel_isr_engine.o(i.uipInterruptServiceEngine) refers to uip_kernel_scheduler.o(.data) for uipNestedInterrupts
    uip_kernel_isr_engine.o(i.uipInterruptServiceEngine) refers to uip_kernel_common.o(.data) for uipLowPowerMode
    uip_kernel_isr_engine.o(i.uipInterruptServiceEngine) refers to uip_kernel_scheduler.o(.data) for uipSchedulerLock
    uip_kernel_isr_engine.o(i.uipInterruptServiceEngine) refers to uip_kernel_scheduler.o(.data) for uipNextRunningTaskTCBPtr
    uip_kernel_message.o(i.UIP_GetMessageStatus) refers to uip_kernel_common.o(.data) for uipMsgNumber
    uip_kernel_message.o(i.UIP_ReadFlag) refers to uip_kernel_common.o(.data) for uipMCBArray
    uip_kernel_message.o(i.UIP_ReceiveMessage) refers to uip_kernel_isr_cm.o(CODE) for uipDisableAllInterrupts
    uip_kernel_message.o(i.UIP_ReceiveMessage) refers to uip_kernel_common.o(.data) for uipMsgNumber
    uip_kernel_message.o(i.UIP_ResetFlag) refers to uip_kernel_isr_cm.o(CODE) for uipDisableAllInterrupts
    uip_kernel_message.o(i.UIP_ResetFlag) refers to uip_kernel_common.o(.data) for uipMCBArray
    uip_kernel_message.o(i.UIP_SendMessage) refers to uip_kernel_isr_cm.o(CODE) for uipDisableAllInterrupts
    uip_kernel_message.o(i.UIP_SendMessage) refers to uip_kernel_event.o(i.UIP_SetEvent) for UIP_SetEvent
    uip_kernel_message.o(i.UIP_SendMessage) refers to uip_kernel_task.o(i.UIP_ActivateTask) for UIP_ActivateTask
    uip_kernel_message.o(i.UIP_SendMessage) refers to uip_kernel_common.o(.data) for uipMsgNumber
    uip_kernel_message.o(i.UIP_StartCOM) refers to demo.o(i.uipCOMInit) for uipCOMInit
    uip_kernel_message.o(i.UIP_StopCOM) refers to uip_kernel_common.o(.data) for uipMCBArray
    uip_kernel_resource.o(i.UIP_GetResource) refers to uip_kernel_isr_cm.o(CODE) for uipDisableAllInterrupts
    uip_kernel_resource.o(i.UIP_GetResource) refers to uip_kernel_scheduler.o(.data) for uipNestedInterrupts
    uip_kernel_resource.o(i.UIP_GetResource) refers to uip_kernel_common.o(.data) for uipResNumber
    uip_kernel_resource.o(i.UIP_GetResource) refers to uip_kernel_scheduler.o(.data) for uipCurrentTaskTCBPtr
    uip_kernel_resource.o(i.UIP_GetResource) refers to uip_kernel_common.o(.bss) for uipPriorityToTaskID
    uip_kernel_resource.o(i.UIP_ReleaseResource) refers to uip_kernel_isr_cm.o(CODE) for uipDisableAllInterrupts
    uip_kernel_resource.o(i.UIP_ReleaseResource) refers to uip_kernel_scheduler.o(i.uipGetNextPriority) for uipGetNextPriority
    uip_kernel_resource.o(i.UIP_ReleaseResource) refers to uip_kernel_common.o(.data) for uipResNumber
    uip_kernel_resource.o(i.UIP_ReleaseResource) refers to uip_kernel_scheduler.o(.data) for uipCurrentTaskTCBPtr
    uip_kernel_resource.o(i.UIP_ReleaseResource) refers to uip_kernel_common.o(.bss) for uipPriorityToTaskID
    uip_kernel_resource.o(i.UIP_ReleaseResource) refers to uip_kernel_scheduler.o(.data) for uipNestedInterrupts
    uip_kernel_scheduler.o(i.uipClearPrioGrpAndArrayBit) refers to uip_kernel_scheduler.o(.data) for .data
    uip_kernel_scheduler.o(i.uipGetNextPriority) refers to uip_kernel_scheduler.o(.data) for .data
    uip_kernel_scheduler.o(i.uipGetNextTask) refers to uip_kernel_scheduler.o(.data) for .data
    uip_kernel_scheduler.o(i.uipGetNextTask) refers to uip_kernel_common.o(.bss) for uipPriorityToTaskID
    uip_kernel_scheduler.o(i.uipGetNextTask) refers to uip_kernel_common.o(.data) for uipTCBArray
    uip_kernel_scheduler.o(i.uipPreContexSwitch) refers to uip_kernel_scheduler.o(i.uipResetPrioGrpAndArrayBit) for uipResetPrioGrpAndArrayBit
    uip_kernel_scheduler.o(i.uipPreContexSwitch) refers to uip_kernel_scheduler.o(.data) for .data
    uip_kernel_scheduler.o(i.uipResetPrioGrpAndArrayBit) refers to uip_kernel_scheduler.o(.data) for .data
    uip_kernel_task.o(i.UIP_ActivateTask) refers to uip_kernel_isr_cm.o(CODE) for uipDisableAllInterrupts
    uip_kernel_task.o(i.UIP_ActivateTask) refers to uip_kernel_common.o(.data) for uipTCBArray
    uip_kernel_task.o(i.UIP_ActivateTask) refers to uip_kernel_scheduler.o(.data) for uipPrioGroup
    uip_kernel_task.o(i.UIP_ActivateTask) refers to uip_kernel_scheduler.o(.data) for uipNestedInterrupts
    uip_kernel_task.o(i.UIP_ActivateTask) refers to uip_kernel_scheduler.o(.data) for uipSchedulerLock
    uip_kernel_task.o(i.UIP_ChainTask) refers to uip_kernel_isr_cm.o(CODE) for uipDisableAllInterrupts
    uip_kernel_task.o(i.UIP_ChainTask) refers to uip_kernel_scheduler.o(i.uipClearPrioGrpAndArrayBit) for uipClearPrioGrpAndArrayBit
    uip_kernel_task.o(i.UIP_ChainTask) refers to uip_kernel_scheduler.o(i.uipGetNextTask) for uipGetNextTask
    uip_kernel_task.o(i.UIP_ChainTask) refers to uip_kernel_common.o(i.uipTaskStackInit) for uipTaskStackInit
    uip_kernel_task.o(i.UIP_ChainTask) refers to uip_kernel_scheduler.o(.data) for uipNestedInterrupts
    uip_kernel_task.o(i.UIP_ChainTask) refers to uip_kernel_scheduler.o(.data) for uipSchedulerLock
    uip_kernel_task.o(i.UIP_ChainTask) refers to uip_kernel_scheduler.o(.data) for uipCurrentTaskTCBPtr
    uip_kernel_task.o(i.UIP_ChainTask) refers to uip_kernel_common.o(.data) for uipTCBArray
    uip_kernel_task.o(i.UIP_ChainTask) refers to uip_kernel_common.o(.bss) for uipInitTaskStackPtr
    uip_kernel_task.o(i.UIP_GetTaskID) refers to uip_kernel_scheduler.o(.data) for uipCurrentTaskTCBPtr
    uip_kernel_task.o(i.UIP_GetTaskState) refers to uip_kernel_isr_cm.o(CODE) for uipDisableAllInterrupts
    uip_kernel_task.o(i.UIP_GetTaskState) refers to uip_kernel_common.o(.data) for uipTCBArray
    uip_kernel_task.o(i.UIP_Schedule) refers to uip_kernel_isr_cm.o(CODE) for uipDisableAllInterrupts
    uip_kernel_task.o(i.UIP_Schedule) refers to uip_kernel_scheduler.o(i.uipGetNextPriority) for uipGetNextPriority
    uip_kernel_task.o(i.UIP_Schedule) refers to uip_kernel_scheduler.o(.data) for uipNestedInterrupts
    uip_kernel_task.o(i.UIP_Schedule) refers to uip_kernel_scheduler.o(.data) for uipSchedulerLock
    uip_kernel_task.o(i.UIP_Schedule) refers to uip_kernel_scheduler.o(.data) for uipCurrentTaskTCBPtr
    uip_kernel_task.o(i.UIP_Schedule) refers to uip_kernel_common.o(.bss) for uipPriorityToTaskID
    uip_kernel_task.o(i.UIP_Schedule) refers to uip_kernel_common.o(.data) for uipTCBArray
    uip_kernel_task.o(i.UIP_TerminateTask) refers to uip_kernel_isr_cm.o(CODE) for uipDisableAllInterrupts
    uip_kernel_task.o(i.UIP_TerminateTask) refers to uip_kernel_common.o(i.uipTaskStackInit) for uipTaskStackInit
    uip_kernel_task.o(i.UIP_TerminateTask) refers to uip_kernel_scheduler.o(i.uipClearPrioGrpAndArrayBit) for uipClearPrioGrpAndArrayBit
    uip_kernel_task.o(i.UIP_TerminateTask) refers to uip_kernel_scheduler.o(i.uipGetNextTask) for uipGetNextTask
    uip_kernel_task.o(i.UIP_TerminateTask) refers to uip_kernel_scheduler.o(.data) for uipNestedInterrupts
    uip_kernel_task.o(i.UIP_TerminateTask) refers to uip_kernel_scheduler.o(.data) for uipSchedulerLock
    uip_kernel_task.o(i.UIP_TerminateTask) refers to uip_kernel_scheduler.o(.data) for uipCurrentTaskTCBPtr
    uip_kernel_task.o(i.UIP_TerminateTask) refers to uip_kernel_common.o(.bss) for uipInitTaskStackPtr
    uip_kernel_time.o(i.UIP_CancelAlarm) refers to uip_kernel_isr_cm.o(CODE) for uipDisableAllInterrupts
    uip_kernel_time.o(i.UIP_CancelAlarm) refers to uip_kernel_common.o(.data) for uipAlarmNumber
    uip_kernel_time.o(i.UIP_GetAlarm) refers to uip_kernel_isr_cm.o(CODE) for uipDisableAllInterrupts
    uip_kernel_time.o(i.UIP_GetAlarm) refers to uip_kernel_common.o(.data) for uipAlarmNumber
    uip_kernel_time.o(i.UIP_GetAlarmBase) refers to uip_kernel_common.o(.data) for uipAlarmNumber
    uip_kernel_time.o(i.UIP_SetAbsAlarm) refers to uip_kernel_isr_cm.o(CODE) for uipDisableAllInterrupts
    uip_kernel_time.o(i.UIP_SetAbsAlarm) refers to uip_kernel_common.o(.data) for uipAlarmNumber
    uip_kernel_time.o(i.UIP_SetRelAlarm) refers to uip_kernel_isr_cm.o(CODE) for uipDisableAllInterrupts
    uip_kernel_time.o(i.UIP_SetRelAlarm) refers to uip_kernel_common.o(.data) for uipAlarmNumber
    uip_kernel_time.o(i.uipAlarmHandler) refers to uip_kernel_event.o(i.UIP_SetEvent) for UIP_SetEvent
    uip_kernel_time.o(i.uipAlarmHandler) refers to uip_kernel_task.o(i.UIP_ActivateTask) for UIP_ActivateTask
    uip_kernel_time.o(i.uipAlarmHandler) refers to uip_kernel_common.o(.data) for uipACBArray
    uip_kernel_time.o(i.uipAlarmHandler) refers to uip_kernel_common.o(.data) for uipIdleTaskID
    uip_kernel_time.o(i.uipGeneralCounterHandler) refers to uip_kernel_time.o(i.uipAlarmHandler) for uipAlarmHandler
    uip_kernel_time.o(i.uipGeneralCounterHandler) refers to uip_kernel_common.o(.data) for uipACBArray
    uip_kernel_time.o(i.uipGetCtrCurrentValue) refers to uip_kernel_isr_cm.o(CODE) for uipDisableAllInterrupts
    uip_kernel_time.o(i.uipGetCtrCurrentValue) refers to uip_kernel_common.o(.data) for uipAlarmNumber
    uip_kernel_time.o(i.uipSystemCounterHandler) refers to uip_kernel_time.o(i.uipAlarmHandler) for uipAlarmHandler
    uip_kernel_time.o(i.uipSystemCounterHandler) refers to uip_kernel_common.o(.bss) for uipSystemCounter
    uip_kernel_time.o(i.uipSystemCounterHandler) refers to uip_kernel_common.o(.data) for uipACBArray
    entry.o(.ARM.Collect$$$$00000000) refers (Special) to entry10a.o(.ARM.Collect$$$$0000000D) for __rt_final_cpp
    entry.o(.ARM.Collect$$$$00000000) refers (Special) to entry11a.o(.ARM.Collect$$$$0000000F) for __rt_final_exit
    entry.o(.ARM.Collect$$$$00000000) refers (Special) to entry7b.o(.ARM.Collect$$$$00000008) for _main_clock
    entry.o(.ARM.Collect$$$$00000000) refers (Special) to entry8b.o(.ARM.Collect$$$$0000000A) for _main_cpp_init
    entry.o(.ARM.Collect$$$$00000000) refers (Special) to entry9a.o(.ARM.Collect$$$$0000000B) for _main_init
    entry.o(.ARM.Collect$$$$00000000) refers (Special) to entry5.o(.ARM.Collect$$$$00000004) for _main_scatterload
    entry.o(.ARM.Collect$$$$00000000) refers (Special) to entry2.o(.ARM.Collect$$$$00000001) for _main_stk
    uldiv.o(.text) refers to llushr.o(.text) for __aeabi_llsr
    uldiv.o(.text) refers to llshl.o(.text) for __aeabi_llsl
    printfb.o(i.__0fprintf$bare) refers to printfb.o(i._printf_core) for _printf_core
    printfb.o(i.__0fprintf$bare) refers to retarget.o(i.fputc) for fputc
    printfb.o(i.__0printf$bare) refers to printfb.o(i._printf_core) for _printf_core
    printfb.o(i.__0printf$bare) refers to retarget.o(i.fputc) for fputc
    printfb.o(i.__0printf$bare) refers to retarget.o(.data) for __stdout
    printfb.o(i.__0snprintf$bare) refers to printfb.o(i._printf_core) for _printf_core
    printfb.o(i.__0snprintf$bare) refers to printfb.o(i._snputc) for _snputc
    printfb.o(i.__0sprintf$bare) refers to printfb.o(i._printf_core) for _printf_core
    printfb.o(i.__0sprintf$bare) refers to printfb.o(i._sputc) for _sputc
    printfb.o(i.__0vfprintf$bare) refers to printfb.o(i._printf_core) for _printf_core
    printfb.o(i.__0vfprintf$bare) refers to retarget.o(i.fputc) for fputc
    printfb.o(i.__0vprintf$bare) refers to printfb.o(i._printf_core) for _printf_core
    printfb.o(i.__0vprintf$bare) refers to retarget.o(i.fputc) for fputc
    printfb.o(i.__0vprintf$bare) refers to retarget.o(.data) for __stdout
    printfb.o(i.__0vsnprintf$bare) refers to printfb.o(i._printf_core) for _printf_core
    printfb.o(i.__0vsnprintf$bare) refers to printfb.o(i._snputc) for _snputc
    printfb.o(i.__0vsprintf$bare) refers to printfb.o(i._printf_core) for _printf_core
    printfb.o(i.__0vsprintf$bare) refers to printfb.o(i._sputc) for _sputc
    printf0.o(i.__0fprintf$0) refers to printf0.o(i._printf_core) for _printf_core
    printf0.o(i.__0fprintf$0) refers to retarget.o(i.fputc) for fputc
    printf0.o(i.__0printf$0) refers to printf0.o(i._printf_core) for _printf_core
    printf0.o(i.__0printf$0) refers to retarget.o(i.fputc) for fputc
    printf0.o(i.__0printf$0) refers to retarget.o(.data) for __stdout
    printf0.o(i.__0snprintf$0) refers to printf0.o(i._printf_core) for _printf_core
    printf0.o(i.__0snprintf$0) refers to printf0.o(i._snputc) for _snputc
    printf0.o(i.__0sprintf$0) refers to printf0.o(i._printf_core) for _printf_core
    printf0.o(i.__0sprintf$0) refers to printf0.o(i._sputc) for _sputc
    printf0.o(i.__0vfprintf$0) refers to printf0.o(i._printf_core) for _printf_core
    printf0.o(i.__0vfprintf$0) refers to retarget.o(i.fputc) for fputc
    printf0.o(i.__0vprintf$0) refers to printf0.o(i._printf_core) for _printf_core
    printf0.o(i.__0vprintf$0) refers to retarget.o(i.fputc) for fputc
    printf0.o(i.__0vprintf$0) refers to retarget.o(.data) for __stdout
    printf0.o(i.__0vsnprintf$0) refers to printf0.o(i._printf_core) for _printf_core
    printf0.o(i.__0vsnprintf$0) refers to printf0.o(i._snputc) for _snputc
    printf0.o(i.__0vsprintf$0) refers to printf0.o(i._printf_core) for _printf_core
    printf0.o(i.__0vsprintf$0) refers to printf0.o(i._sputc) for _sputc
    printf1.o(i.__0fprintf$1) refers to printf1.o(i._printf_core) for _printf_core
    printf1.o(i.__0fprintf$1) refers to retarget.o(i.fputc) for fputc
    printf1.o(i.__0printf$1) refers to printf1.o(i._printf_core) for _printf_core
    printf1.o(i.__0printf$1) refers to retarget.o(i.fputc) for fputc
    printf1.o(i.__0printf$1) refers to retarget.o(.data) for __stdout
    printf1.o(i.__0snprintf$1) refers to printf1.o(i._printf_core) for _printf_core
    printf1.o(i.__0snprintf$1) refers to printf1.o(i._snputc) for _snputc
    printf1.o(i.__0sprintf$1) refers to printf1.o(i._printf_core) for _printf_core
    printf1.o(i.__0sprintf$1) refers to printf1.o(i._sputc) for _sputc
    printf1.o(i.__0vfprintf$1) refers to printf1.o(i._printf_core) for _printf_core
    printf1.o(i.__0vfprintf$1) refers to retarget.o(i.fputc) for fputc
    printf1.o(i.__0vprintf$1) refers to printf1.o(i._printf_core) for _printf_core
    printf1.o(i.__0vprintf$1) refers to retarget.o(i.fputc) for fputc
    printf1.o(i.__0vprintf$1) refers to retarget.o(.data) for __stdout
    printf1.o(i.__0vsnprintf$1) refers to printf1.o(i._printf_core) for _printf_core
    printf1.o(i.__0vsnprintf$1) refers to printf1.o(i._snputc) for _snputc
    printf1.o(i.__0vsprintf$1) refers to printf1.o(i._printf_core) for _printf_core
    printf1.o(i.__0vsprintf$1) refers to printf1.o(i._sputc) for _sputc
    printf1.o(i._printf_core) refers to uidiv.o(.text) for __aeabi_uidivmod
    printf2.o(i.__0fprintf$2) refers to printf2.o(i._printf_core) for _printf_core
    printf2.o(i.__0fprintf$2) refers to retarget.o(i.fputc) for fputc
    printf2.o(i.__0printf$2) refers to printf2.o(i._printf_core) for _printf_core
    printf2.o(i.__0printf$2) refers to retarget.o(i.fputc) for fputc
    printf2.o(i.__0printf$2) refers to retarget.o(.data) for __stdout
    printf2.o(i.__0snprintf$2) refers to printf2.o(i._printf_core) for _printf_core
    printf2.o(i.__0snprintf$2) refers to printf2.o(i._snputc) for _snputc
    printf2.o(i.__0sprintf$2) refers to printf2.o(i._printf_core) for _printf_core
    printf2.o(i.__0sprintf$2) refers to printf2.o(i._sputc) for _sputc
    printf2.o(i.__0vfprintf$2) refers to printf2.o(i._printf_core) for _printf_core
    printf2.o(i.__0vfprintf$2) refers to retarget.o(i.fputc) for fputc
    printf2.o(i.__0vprintf$2) refers to printf2.o(i._printf_core) for _printf_core
    printf2.o(i.__0vprintf$2) refers to retarget.o(i.fputc) for fputc
    printf2.o(i.__0vprintf$2) refers to retarget.o(.data) for __stdout
    printf2.o(i.__0vsnprintf$2) refers to printf2.o(i._printf_core) for _printf_core
    printf2.o(i.__0vsnprintf$2) refers to printf2.o(i._snputc) for _snputc
    printf2.o(i.__0vsprintf$2) refers to printf2.o(i._printf_core) for _printf_core
    printf2.o(i.__0vsprintf$2) refers to printf2.o(i._sputc) for _sputc
    printf3.o(i.__0fprintf$3) refers to printf3.o(i._printf_core) for _printf_core
    printf3.o(i.__0fprintf$3) refers to retarget.o(i.fputc) for fputc
    printf3.o(i.__0printf$3) refers to printf3.o(i._printf_core) for _printf_core
    printf3.o(i.__0printf$3) refers to retarget.o(i.fputc) for fputc
    printf3.o(i.__0printf$3) refers to retarget.o(.data) for __stdout
    printf3.o(i.__0snprintf$3) refers to printf3.o(i._printf_core) for _printf_core
    printf3.o(i.__0snprintf$3) refers to printf3.o(i._snputc) for _snputc
    printf3.o(i.__0sprintf$3) refers to printf3.o(i._printf_core) for _printf_core
    printf3.o(i.__0sprintf$3) refers to printf3.o(i._sputc) for _sputc
    printf3.o(i.__0vfprintf$3) refers to printf3.o(i._printf_core) for _printf_core
    printf3.o(i.__0vfprintf$3) refers to retarget.o(i.fputc) for fputc
    printf3.o(i.__0vprintf$3) refers to printf3.o(i._printf_core) for _printf_core
    printf3.o(i.__0vprintf$3) refers to retarget.o(i.fputc) for fputc
    printf3.o(i.__0vprintf$3) refers to retarget.o(.data) for __stdout
    printf3.o(i.__0vsnprintf$3) refers to printf3.o(i._printf_core) for _printf_core
    printf3.o(i.__0vsnprintf$3) refers to printf3.o(i._snputc) for _snputc
    printf3.o(i.__0vsprintf$3) refers to printf3.o(i._printf_core) for _printf_core
    printf3.o(i.__0vsprintf$3) refers to printf3.o(i._sputc) for _sputc
    printf3.o(i._printf_core) refers to uidiv.o(.text) for __aeabi_uidivmod
    printf4.o(i.__0fprintf$4) refers to printf4.o(i._printf_core) for _printf_core
    printf4.o(i.__0fprintf$4) refers to retarget.o(i.fputc) for fputc
    printf4.o(i.__0printf$4) refers to printf4.o(i._printf_core) for _printf_core
    printf4.o(i.__0printf$4) refers to retarget.o(i.fputc) for fputc
    printf4.o(i.__0printf$4) refers to retarget.o(.data) for __stdout
    printf4.o(i.__0snprintf$4) refers to printf4.o(i._printf_core) for _printf_core
    printf4.o(i.__0snprintf$4) refers to printf4.o(i._snputc) for _snputc
    printf4.o(i.__0sprintf$4) refers to printf4.o(i._printf_core) for _printf_core
    printf4.o(i.__0sprintf$4) refers to printf4.o(i._sputc) for _sputc
    printf4.o(i.__0vfprintf$4) refers to printf4.o(i._printf_core) for _printf_core
    printf4.o(i.__0vfprintf$4) refers to retarget.o(i.fputc) for fputc
    printf4.o(i.__0vprintf$4) refers to printf4.o(i._printf_core) for _printf_core
    printf4.o(i.__0vprintf$4) refers to retarget.o(i.fputc) for fputc
    printf4.o(i.__0vprintf$4) refers to retarget.o(.data) for __stdout
    printf4.o(i.__0vsnprintf$4) refers to printf4.o(i._printf_core) for _printf_core
    printf4.o(i.__0vsnprintf$4) refers to printf4.o(i._snputc) for _snputc
    printf4.o(i.__0vsprintf$4) refers to printf4.o(i._printf_core) for _printf_core
    printf4.o(i.__0vsprintf$4) refers to printf4.o(i._sputc) for _sputc
    printf4.o(i._printf_core) refers to uldiv.o(.text) for __aeabi_uldivmod
    printf5.o(i.__0fprintf$5) refers to printf5.o(i._printf_core) for _printf_core
    printf5.o(i.__0fprintf$5) refers to retarget.o(i.fputc) for fputc
    printf5.o(i.__0printf$5) refers to printf5.o(i._printf_core) for _printf_core
    printf5.o(i.__0printf$5) refers to retarget.o(i.fputc) for fputc
    printf5.o(i.__0printf$5) refers to retarget.o(.data) for __stdout
    printf5.o(i.__0snprintf$5) refers to printf5.o(i._printf_core) for _printf_core
    printf5.o(i.__0snprintf$5) refers to printf5.o(i._snputc) for _snputc
    printf5.o(i.__0sprintf$5) refers to printf5.o(i._printf_core) for _printf_core
    printf5.o(i.__0sprintf$5) refers to printf5.o(i._sputc) for _sputc
    printf5.o(i.__0vfprintf$5) refers to printf5.o(i._printf_core) for _printf_core
    printf5.o(i.__0vfprintf$5) refers to retarget.o(i.fputc) for fputc
    printf5.o(i.__0vprintf$5) refers to printf5.o(i._printf_core) for _printf_core
    printf5.o(i.__0vprintf$5) refers to retarget.o(i.fputc) for fputc
    printf5.o(i.__0vprintf$5) refers to retarget.o(.data) for __stdout
    printf5.o(i.__0vsnprintf$5) refers to printf5.o(i._printf_core) for _printf_core
    printf5.o(i.__0vsnprintf$5) refers to printf5.o(i._snputc) for _snputc
    printf5.o(i.__0vsprintf$5) refers to printf5.o(i._printf_core) for _printf_core
    printf5.o(i.__0vsprintf$5) refers to printf5.o(i._sputc) for _sputc
    printf5.o(i._printf_core) refers to uldiv.o(.text) for __aeabi_uldivmod
    printf6.o(i.__0fprintf$6) refers to printf6.o(i._printf_core) for _printf_core
    printf6.o(i.__0fprintf$6) refers to retarget.o(i.fputc) for fputc
    printf6.o(i.__0printf$6) refers to printf6.o(i._printf_core) for _printf_core
    printf6.o(i.__0printf$6) refers to retarget.o(i.fputc) for fputc
    printf6.o(i.__0printf$6) refers to retarget.o(.data) for __stdout
    printf6.o(i.__0snprintf$6) refers to printf6.o(i._printf_core) for _printf_core
    printf6.o(i.__0snprintf$6) refers to printf6.o(i._snputc) for _snputc
    printf6.o(i.__0sprintf$6) refers to printf6.o(i._printf_core) for _printf_core
    printf6.o(i.__0sprintf$6) refers to printf6.o(i._sputc) for _sputc
    printf6.o(i.__0vfprintf$6) refers to printf6.o(i._printf_core) for _printf_core
    printf6.o(i.__0vfprintf$6) refers to retarget.o(i.fputc) for fputc
    printf6.o(i.__0vprintf$6) refers to printf6.o(i._printf_core) for _printf_core
    printf6.o(i.__0vprintf$6) refers to retarget.o(i.fputc) for fputc
    printf6.o(i.__0vprintf$6) refers to retarget.o(.data) for __stdout
    printf6.o(i.__0vsnprintf$6) refers to printf6.o(i._printf_core) for _printf_core
    printf6.o(i.__0vsnprintf$6) refers to printf6.o(i._snputc) for _snputc
    printf6.o(i.__0vsprintf$6) refers to printf6.o(i._printf_core) for _printf_core
    printf6.o(i.__0vsprintf$6) refers to printf6.o(i._sputc) for _sputc
    printf6.o(i._printf_core) refers to printf6.o(i._printf_pre_padding) for _printf_pre_padding
    printf6.o(i._printf_core) refers to printf6.o(i._printf_post_padding) for _printf_post_padding
    printf6.o(i._printf_core) refers to uidiv.o(.text) for __aeabi_uidivmod
    printf7.o(i.__0fprintf$7) refers to printf7.o(i._printf_core) for _printf_core
    printf7.o(i.__0fprintf$7) refers to retarget.o(i.fputc) for fputc
    printf7.o(i.__0printf$7) refers to printf7.o(i._printf_core) for _printf_core
    printf7.o(i.__0printf$7) refers to retarget.o(i.fputc) for fputc
    printf7.o(i.__0printf$7) refers to retarget.o(.data) for __stdout
    printf7.o(i.__0snprintf$7) refers to printf7.o(i._printf_core) for _printf_core
    printf7.o(i.__0snprintf$7) refers to printf7.o(i._snputc) for _snputc
    printf7.o(i.__0sprintf$7) refers to printf7.o(i._printf_core) for _printf_core
    printf7.o(i.__0sprintf$7) refers to printf7.o(i._sputc) for _sputc
    printf7.o(i.__0vfprintf$7) refers to printf7.o(i._printf_core) for _printf_core
    printf7.o(i.__0vfprintf$7) refers to retarget.o(i.fputc) for fputc
    printf7.o(i.__0vprintf$7) refers to printf7.o(i._printf_core) for _printf_core
    printf7.o(i.__0vprintf$7) refers to retarget.o(i.fputc) for fputc
    printf7.o(i.__0vprintf$7) refers to retarget.o(.data) for __stdout
    printf7.o(i.__0vsnprintf$7) refers to printf7.o(i._printf_core) for _printf_core
    printf7.o(i.__0vsnprintf$7) refers to printf7.o(i._snputc) for _snputc
    printf7.o(i.__0vsprintf$7) refers to printf7.o(i._printf_core) for _printf_core
    printf7.o(i.__0vsprintf$7) refers to printf7.o(i._sputc) for _sputc
    printf7.o(i._printf_core) refers to printf7.o(i._printf_pre_padding) for _printf_pre_padding
    printf7.o(i._printf_core) refers to printf7.o(i._printf_post_padding) for _printf_post_padding
    printf7.o(i._printf_core) refers to uldiv.o(.text) for __aeabi_uldivmod
    printf8.o(i.__0fprintf$8) refers to printf8.o(i._printf_core) for _printf_core
    printf8.o(i.__0fprintf$8) refers to retarget.o(i.fputc) for fputc
    printf8.o(i.__0printf$8) refers to printf8.o(i._printf_core) for _printf_core
    printf8.o(i.__0printf$8) refers to retarget.o(i.fputc) for fputc
    printf8.o(i.__0printf$8) refers to retarget.o(.data) for __stdout
    printf8.o(i.__0snprintf$8) refers to printf8.o(i._printf_core) for _printf_core
    printf8.o(i.__0snprintf$8) refers to printf8.o(i._snputc) for _snputc
    printf8.o(i.__0sprintf$8) refers to printf8.o(i._printf_core) for _printf_core
    printf8.o(i.__0sprintf$8) refers to printf8.o(i._sputc) for _sputc
    printf8.o(i.__0vfprintf$8) refers to printf8.o(i._printf_core) for _printf_core
    printf8.o(i.__0vfprintf$8) refers to retarget.o(i.fputc) for fputc
    printf8.o(i.__0vprintf$8) refers to printf8.o(i._printf_core) for _printf_core
    printf8.o(i.__0vprintf$8) refers to retarget.o(i.fputc) for fputc
    printf8.o(i.__0vprintf$8) refers to retarget.o(.data) for __stdout
    printf8.o(i.__0vsnprintf$8) refers to printf8.o(i._printf_core) for _printf_core
    printf8.o(i.__0vsnprintf$8) refers to printf8.o(i._snputc) for _snputc
    printf8.o(i.__0vsprintf$8) refers to printf8.o(i._printf_core) for _printf_core
    printf8.o(i.__0vsprintf$8) refers to printf8.o(i._sputc) for _sputc
    printf8.o(i._printf_core) refers to printf8.o(i._printf_pre_padding) for _printf_pre_padding
    printf8.o(i._printf_core) refers to printf8.o(i._printf_post_padding) for _printf_post_padding
    printf8.o(i._printf_core) refers to uldiv.o(.text) for __aeabi_uldivmod
    printfa.o(i.__0fprintf) refers (Special) to iusefp.o(.text) for __I$use$fp
    printfa.o(i.__0fprintf) refers to printfa.o(i._printf_core) for _printf_core
    printfa.o(i.__0fprintf) refers to retarget.o(i.fputc) for fputc
    printfa.o(i.__0printf) refers (Special) to iusefp.o(.text) for __I$use$fp
    printfa.o(i.__0printf) refers to printfa.o(i._printf_core) for _printf_core
    printfa.o(i.__0printf) refers to retarget.o(i.fputc) for fputc
    printfa.o(i.__0printf) refers to retarget.o(.data) for __stdout
    printfa.o(i.__0snprintf) refers (Special) to iusefp.o(.text) for __I$use$fp
    printfa.o(i.__0snprintf) refers to printfa.o(i._printf_core) for _printf_core
    printfa.o(i.__0snprintf) refers to printfa.o(i._snputc) for _snputc
    printfa.o(i.__0sprintf) refers (Special) to iusefp.o(.text) for __I$use$fp
    printfa.o(i.__0sprintf) refers to printfa.o(i._printf_core) for _printf_core
    printfa.o(i.__0sprintf) refers to printfa.o(i._sputc) for _sputc
    printfa.o(i.__0vfprintf) refers (Special) to iusefp.o(.text) for __I$use$fp
    printfa.o(i.__0vfprintf) refers to printfa.o(i._printf_core) for _printf_core
    printfa.o(i.__0vfprintf) refers to retarget.o(i.fputc) for fputc
    printfa.o(i.__0vprintf) refers (Special) to iusefp.o(.text) for __I$use$fp
    printfa.o(i.__0vprintf) refers to printfa.o(i._printf_core) for _printf_core
    printfa.o(i.__0vprintf) refers to retarget.o(i.fputc) for fputc
    printfa.o(i.__0vprintf) refers to retarget.o(.data) for __stdout
    printfa.o(i.__0vsnprintf) refers (Special) to iusefp.o(.text) for __I$use$fp
    printfa.o(i.__0vsnprintf) refers to printfa.o(i._printf_core) for _printf_core
    printfa.o(i.__0vsnprintf) refers to printfa.o(i._snputc) for _snputc
    printfa.o(i.__0vsprintf) refers (Special) to iusefp.o(.text) for __I$use$fp
    printfa.o(i.__0vsprintf) refers to printfa.o(i._printf_core) for _printf_core
    printfa.o(i.__0vsprintf) refers to printfa.o(i._sputc) for _sputc
    printfa.o(i._fp_digits) refers (Special) to iusefp.o(.text) for __I$use$fp
    printfa.o(i._fp_digits) refers to dmul.o(.text) for __aeabi_dmul
    printfa.o(i._fp_digits) refers to ddiv.o(.text) for __aeabi_ddiv
    printfa.o(i._fp_digits) refers to cdrcmple.o(.text) for __aeabi_cdrcmple
    printfa.o(i._fp_digits) refers to dadd.o(.text) for __aeabi_dadd
    printfa.o(i._fp_digits) refers to dfixul.o(.text) for __aeabi_d2ulz
    printfa.o(i._fp_digits) refers to uldiv.o(.text) for __aeabi_uldivmod
    printfa.o(i._printf_core) refers (Special) to iusefp.o(.text) for __I$use$fp
    printfa.o(i._printf_core) refers to printfa.o(i._printf_pre_padding) for _printf_pre_padding
    printfa.o(i._printf_core) refers to uldiv.o(.text) for __aeabi_uldivmod
    printfa.o(i._printf_core) refers to printfa.o(i._printf_post_padding) for _printf_post_padding
    printfa.o(i._printf_core) refers to printfa.o(i._fp_digits) for _fp_digits
    printfa.o(i._printf_core) refers to uidiv.o(.text) for __aeabi_uidivmod
    printfa.o(i._printf_post_padding) refers (Special) to iusefp.o(.text) for __I$use$fp
    printfa.o(i._printf_pre_padding) refers (Special) to iusefp.o(.text) for __I$use$fp
    printfa.o(i._snputc) refers (Special) to iusefp.o(.text) for __I$use$fp
    printfa.o(i._sputc) refers (Special) to iusefp.o(.text) for __I$use$fp
    atoi.o(.text) refers to errno.o(i.__aeabi_errno_addr) for __aeabi_errno_addr
    atoi.o(.text) refers to strtol.o(.text) for strtol
    entry2.o(.ARM.Collect$$$$00000001) refers to entry2.o(.ARM.Collect$$$$00002712) for __lit__00000000
    entry2.o(.ARM.Collect$$$$00002712) refers to startup_nuc200series.o(STACK) for __initial_sp
    entry2.o(__vectab_stack_and_reset_area) refers to startup_nuc200series.o(STACK) for __initial_sp
    entry2.o(__vectab_stack_and_reset_area) refers to entry.o(.ARM.Collect$$$$00000000) for __main
    entry5.o(.ARM.Collect$$$$00000004) refers to init.o(.text) for __scatterload
    entry9a.o(.ARM.Collect$$$$0000000B) refers to demo.o(i.main) for main
    entry9b.o(.ARM.Collect$$$$0000000C) refers to demo.o(i.main) for main
    errno.o(i.__aeabi_errno_addr) refers to errno.o(.data) for .data
    errno.o(i.__read_errno) refers to errno.o(.data) for .data
    errno.o(i.__set_errno) refers to errno.o(.data) for .data
    strtol.o(.text) refers to ctype_o.o(.text) for __rt_ctype_table
    strtol.o(.text) refers to _strtoul.o(.text) for _strtoul
    strtol.o(.text) refers to errno.o(i.__aeabi_errno_addr) for __aeabi_errno_addr
    dadd.o(.text) refers to llshl.o(.text) for __aeabi_llsl
    dadd.o(.text) refers to llsshr.o(.text) for __aeabi_lasr
    dadd.o(.text) refers to depilogue.o(.text) for _double_epilogue
    dmul.o(.text) refers to depilogue.o(.text) for _double_epilogue
    ddiv.o(.text) refers to depilogue.o(.text) for _double_round
    dfixul.o(.text) refers to llushr.o(.text) for __aeabi_llsr
    dfixul.o(.text) refers to llshl.o(.text) for __aeabi_llsl
    init.o(.text) refers to entry5.o(.ARM.Collect$$$$00000004) for __main_after_scatterload
    ctype_o.o(.text) refers to ctype_o.o(.constdata) for .constdata
    ctype_o.o(.constdata) refers to ctype_o.o(.constdata) for __ctype_table
    isalnum_o.o(.text) refers to ctype_o.o(.text) for __rt_ctype_table
    isalpha_o.o(.text) refers to ctype_o.o(.text) for __rt_ctype_table
    isblank_o.o(.text) refers to ctype_o.o(.constdata) for __ctype_table
    iscntrl_o.o(.text) refers to ctype_o.o(.text) for __rt_ctype_table
    isdigit_o.o(.text) refers to ctype_o.o(.text) for __rt_ctype_table
    isgraph_o.o(.text) refers to ctype_o.o(.text) for __rt_ctype_table
    islower_o.o(.text) refers to ctype_o.o(.text) for __rt_ctype_table
    isprint_o.o(.text) refers to ctype_o.o(.text) for __rt_ctype_table
    ispunct_o.o(.text) refers to ctype_o.o(.text) for __rt_ctype_table
    isspace_o.o(.text) refers to ctype_o.o(.text) for __rt_ctype_table
    isupper_o.o(.text) refers to ctype_o.o(.text) for __rt_ctype_table
    isxdigit_o.o(.text) refers to ctype_o.o(.text) for __rt_ctype_table
    _strtoul.o(.text) refers to _chval.o(.text) for _chval
    _strtoul.o(.text) refers to errno.o(i.__aeabi_errno_addr) for __aeabi_errno_addr
    depilogue.o(.text) refers to depilogue.o(i.__ARM_clz) for __ARM_clz
    depilogue.o(.text) refers to llshl.o(.text) for __aeabi_llsl
    depilogue.o(.text) refers to llushr.o(.text) for __aeabi_llsr


==============================================================================

Removing Unused input sections from the image.

    Removing system_nuc200series.o(.rev16_text), (4 bytes).
    Removing system_nuc200series.o(.revsh_text), (4 bytes).
    Removing startup_nuc200series.o(HEAP), (0 bytes).
    Removing demo.o(.rev16_text), (4 bytes).
    Removing demo.o(.revsh_text), (4 bytes).
    Removing demo.o(i.uipCOMInit), (4 bytes).
    Removing hook.o(i.COMErrorHook), (2 bytes).
    Removing hook.o(i.ErrorHook), (2 bytes).
    Removing hook.o(i.PostTaskHook), (2 bytes).
    Removing hook.o(i.PreTaskHook), (2 bytes).
    Removing hook.o(i.ShutdownHook), (2 bytes).
    Removing hook.o(i.StuipCOMExtension), (4 bytes).
    Removing hook.o(i.StuipupHook), (2 bytes).
    Removing init.o(.rev16_text), (4 bytes).
    Removing init.o(.revsh_text), (4 bytes).
    Removing retarget.o(.rev16_text), (4 bytes).
    Removing retarget.o(.revsh_text), (4 bytes).
    Removing retarget.o(i.GetChar), (20 bytes).
    Removing retarget.o(i.IsDebugFifoEmpty), (16 bytes).
    Removing retarget.o(i.SendChar), (8 bytes).
    Removing retarget.o(i._ttywrch), (8 bytes).
    Removing retarget.o(i.ferror), (6 bytes).
    Removing retarget.o(i.fgetc), (8 bytes).
    Removing retarget.o(i.kbhit), (16 bytes).
    Removing retarget.o(.data), (4 bytes).
    Removing clk.o(.rev16_text), (4 bytes).
    Removing clk.o(.revsh_text), (4 bytes).
    Removing clk.o(i.CLK_DisableCKO), (16 bytes).
    Removing clk.o(i.CLK_DisableModuleClock), (48 bytes).
    Removing clk.o(i.CLK_DisablePLL), (16 bytes).
    Removing clk.o(i.CLK_DisableSysTick), (12 bytes).
    Removing clk.o(i.CLK_DisableXtalRC), (16 bytes).
    Removing clk.o(i.CLK_EnableCKO), (40 bytes).
    Removing clk.o(i.CLK_EnableSysTick), (56 bytes).
    Removing clk.o(i.CLK_GetCPUFreq), (16 bytes).
    Removing clk.o(i.CLK_GetHCLKFreq), (16 bytes).
    Removing clk.o(i.CLK_GetHXTFreq), (20 bytes).
    Removing clk.o(i.CLK_GetLXTFreq), (24 bytes).
    Removing clk.o(i.CLK_GetPCLKFreq), (16 bytes).
    Removing clk.o(i.CLK_Idle), (32 bytes).
    Removing clk.o(i.CLK_PowerDown), (36 bytes).
    Removing clk.o(i.CLK_SetSysTickClockSrc), (20 bytes).
    Removing sys.o(.rev16_text), (4 bytes).
    Removing sys.o(.revsh_text), (4 bytes).
    Removing sys.o(i.SYS_ClearResetSrc), (12 bytes).
    Removing sys.o(i.SYS_DisableBOD), (14 bytes).
    Removing sys.o(i.SYS_EnableBOD), (36 bytes).
    Removing sys.o(i.SYS_GetBODStatus), (12 bytes).
    Removing sys.o(i.SYS_GetResetSrc), (8 bytes).
    Removing sys.o(i.SYS_IsRegLocked), (16 bytes).
    Removing sys.o(i.SYS_ReadPDID), (8 bytes).
    Removing sys.o(i.SYS_ResetCPU), (14 bytes).
    Removing sys.o(i.SYS_ResetChip), (14 bytes).
    Removing uart.o(.rev16_text), (4 bytes).
    Removing uart.o(.revsh_text), (4 bytes).
    Removing uart.o(i.UART_ClearIntFlag), (56 bytes).
    Removing uart.o(i.UART_Close), (6 bytes).
    Removing uart.o(i.UART_DisableFlowCtrl), (12 bytes).
    Removing uart.o(i.UART_DisableInt), (48 bytes).
    Removing uart.o(i.UART_EnableFlowCtrl), (30 bytes).
    Removing uart.o(i.UART_EnableInt), (48 bytes).
    Removing uart.o(i.UART_Read), (44 bytes).
    Removing uart.o(i.UART_SelectIrDAMode), (132 bytes).
    Removing uart.o(i.UART_SelectLINMode), (24 bytes).
    Removing uart.o(i.UART_SelectRS485Mode), (32 bytes).
    Removing uart.o(i.UART_SetLine_Config), (128 bytes).
    Removing uart.o(i.UART_SetTimeoutCnt), (22 bytes).
    Removing uart.o(i.UART_Write), (44 bytes).
    Removing adc.o(.rev16_text), (4 bytes).
    Removing adc.o(.revsh_text), (4 bytes).
    Removing adc.o(i.ADC_Close), (10 bytes).
    Removing adc.o(i.ADC_DisableHWTrigger), (12 bytes).
    Removing adc.o(i.ADC_EnableHWTrigger), (28 bytes).
    Removing chip_uip_interrupt.o(i.Chip_UIP_InterruptInit), (44 bytes).
    Removing chip_uip_interrupt.o(i.Chip_UIP_InterruptNullHandler), (2 bytes).
    Removing chip_uip_interrupt.o(i.Chip_UIP_InterruptRegisterHandler), (20 bytes).
    Removing chip_uip_interrupt.o(i.Chip_UIP_InterruptRemoveHandler), (20 bytes).
    Removing chip_uip_interrupt.o(i.Chip_UIP_Kernel_Tick_ISR_Handler), (8 bytes).
    Removing chip_uip_interrupt.o(i.Chip_UIP_Kernel_Tick_ISR_Handler_Callback), (4 bytes).
    Removing hardware_init.o(.rev16_text), (4 bytes).
    Removing hardware_init.o(.revsh_text), (4 bytes).
    Removing uip_kernel_common.o(i.ShutdownOS), (2 bytes).
    Removing uip_kernel_common.o(i.uipAlarmInfoInit), (12 bytes).
    Removing uip_kernel_common.o(i.uipMsgInfoInit), (12 bytes).
    Removing uip_kernel_common.o(i.uipResInfoInit), (12 bytes).
    Removing uip_kernel_common.o(i.uipTaskInfoInit), (12 bytes).
    Removing uip_kernel_common.o(.data), (1 bytes).
    Removing uip_kernel_common.o(.data), (4 bytes).
    Removing uip_kernel_event.o(i.UIP_GetEvent), (96 bytes).
    Removing uip_kernel_message.o(i.UIP_CloseCOM), (4 bytes).
    Removing uip_kernel_message.o(i.UIP_GetMessageStatus), (72 bytes).
    Removing uip_kernel_message.o(i.UIP_ReadFlag), (20 bytes).
    Removing uip_kernel_message.o(i.UIP_ResetFlag), (32 bytes).
    Removing uip_kernel_message.o(i.UIP_StartCOM), (8 bytes).
    Removing uip_kernel_message.o(i.UIP_StopCOM), (48 bytes).
    Removing uip_kernel_scheduler.o(.data), (1 bytes).
    Removing uip_kernel_scheduler.o(.data), (1 bytes).
    Removing uip_kernel_task.o(i.UIP_ChainTask), (328 bytes).
    Removing uip_kernel_task.o(i.UIP_GetTaskID), (24 bytes).
    Removing uip_kernel_task.o(i.UIP_GetTaskState), (52 bytes).
    Removing uip_kernel_task.o(i.UIP_Schedule), (232 bytes).
    Removing uip_kernel_time.o(i.UIP_CancelAlarm), (64 bytes).
    Removing uip_kernel_time.o(i.UIP_GetAlarm), (84 bytes).
    Removing uip_kernel_time.o(i.UIP_GetAlarmBase), (20 bytes).
    Removing uip_kernel_time.o(i.UIP_SetAbsAlarm), (104 bytes).
    Removing uip_kernel_time.o(i.UIP_SetRelAlarm), (120 bytes).
    Removing uip_kernel_time.o(i.uipAlarmHandler), (92 bytes).
    Removing uip_kernel_time.o(i.uipGeneralCounterHandler), (72 bytes).
    Removing uip_kernel_time.o(i.uipGetCtrCurrentValue), (68 bytes).
    Removing uip_kernel_time.o(i.uipSystemCounterHandler), (104 bytes).
    Removing dadd.o(.text), (356 bytes).
    Removing dmul.o(.text), (208 bytes).
    Removing ddiv.o(.text), (240 bytes).
    Removing dfixul.o(.text), (64 bytes).
    Removing cdrcmple.o(.text), (40 bytes).
    Removing depilogue.o(.text), (190 bytes).
    Removing depilogue.o(i.__ARM_clz), (46 bytes).

117 unused section(s) (total 4315 bytes) removed from the image.

==============================================================================

Image Symbol Table

    Local Symbols

    Symbol Name                              Value     Ov Type        Size  Object(Section)

    RESET                                    0x00000000   Section      192  startup_nuc200series.o(RESET)
    ../clib/microlib/ctype/ctype.c           0x00000000   Number         0  iscntrl_o.o ABSOLUTE
    ../clib/microlib/ctype/ctype.c           0x00000000   Number         0  isalnum_o.o ABSOLUTE
    ../clib/microlib/ctype/ctype.c           0x00000000   Number         0  isblank_o.o ABSOLUTE
    ../clib/microlib/ctype/ctype.c           0x00000000   Number         0  isalpha_o.o ABSOLUTE
    ../clib/microlib/ctype/ctype.c           0x00000000   Number         0  ctype_o.o ABSOLUTE
    ../clib/microlib/ctype/ctype.c           0x00000000   Number         0  isxdigit_o.o ABSOLUTE
    ../clib/microlib/ctype/ctype.c           0x00000000   Number         0  isupper_o.o ABSOLUTE
    ../clib/microlib/ctype/ctype.c           0x00000000   Number         0  isspace_o.o ABSOLUTE
    ../clib/microlib/ctype/ctype.c           0x00000000   Number         0  ispunct_o.o ABSOLUTE
    ../clib/microlib/ctype/ctype.c           0x00000000   Number         0  isprint_o.o ABSOLUTE
    ../clib/microlib/ctype/ctype.c           0x00000000   Number         0  islower_o.o ABSOLUTE
    ../clib/microlib/ctype/ctype.c           0x00000000   Number         0  isgraph_o.o ABSOLUTE
    ../clib/microlib/ctype/ctype.c           0x00000000   Number         0  isdigit_o.o ABSOLUTE
    ../clib/microlib/division.c              0x00000000   Number         0  uldiv.o ABSOLUTE
    ../clib/microlib/division.c              0x00000000   Number         0  uidiv.o ABSOLUTE
    ../clib/microlib/errno.c                 0x00000000   Number         0  errno.o ABSOLUTE
    ../clib/microlib/init/entry.s            0x00000000   Number         0  entry9b.o ABSOLUTE
    ../clib/microlib/init/entry.s            0x00000000   Number         0  entry9a.o ABSOLUTE
    ../clib/microlib/init/entry.s            0x00000000   Number         0  entry8b.o ABSOLUTE
    ../clib/microlib/init/entry.s            0x00000000   Number         0  entry8a.o ABSOLUTE
    ../clib/microlib/init/entry.s            0x00000000   Number         0  entry11b.o ABSOLUTE
    ../clib/microlib/init/entry.s            0x00000000   Number         0  entry2.o ABSOLUTE
    ../clib/microlib/init/entry.s            0x00000000   Number         0  entry7b.o ABSOLUTE
    ../clib/microlib/init/entry.s            0x00000000   Number         0  entry7a.o ABSOLUTE
    ../clib/microlib/init/entry.s            0x00000000   Number         0  entry10a.o ABSOLUTE
    ../clib/microlib/init/entry.s            0x00000000   Number         0  entry11a.o ABSOLUTE
    ../clib/microlib/init/entry.s            0x00000000   Number         0  entry10b.o ABSOLUTE
    ../clib/microlib/init/entry.s            0x00000000   Number         0  entry5.o ABSOLUTE
    ../clib/microlib/init/entry.s            0x00000000   Number         0  entry.o ABSOLUTE
    ../clib/microlib/longlong.c              0x00000000   Number         0  llushr.o ABSOLUTE
    ../clib/microlib/longlong.c              0x00000000   Number         0  llshl.o ABSOLUTE
    ../clib/microlib/longlong.c              0x00000000   Number         0  llsshr.o ABSOLUTE
    ../clib/microlib/printf/printf.c         0x00000000   Number         0  printf3.o ABSOLUTE
    ../clib/microlib/printf/printf.c         0x00000000   Number         0  printf1.o ABSOLUTE
    ../clib/microlib/printf/printf.c         0x00000000   Number         0  printf0.o ABSOLUTE
    ../clib/microlib/printf/printf.c         0x00000000   Number         0  printf2.o ABSOLUTE
    ../clib/microlib/printf/printf.c         0x00000000   Number         0  printf4.o ABSOLUTE
    ../clib/microlib/printf/printf.c         0x00000000   Number         0  printf5.o ABSOLUTE
    ../clib/microlib/printf/printf.c         0x00000000   Number         0  printf6.o ABSOLUTE
    ../clib/microlib/printf/printf.c         0x00000000   Number         0  printfb.o ABSOLUTE
    ../clib/microlib/printf/printf.c         0x00000000   Number         0  printf7.o ABSOLUTE
    ../clib/microlib/printf/printf.c         0x00000000   Number         0  printf8.o ABSOLUTE
    ../clib/microlib/printf/printf.c         0x00000000   Number         0  printfa.o ABSOLUTE
    ../clib/microlib/printf/stubs.s          0x00000000   Number         0  stubs.o ABSOLUTE
    ../clib/microlib/stubs.s                 0x00000000   Number         0  iusefp.o ABSOLUTE
    ../clib/scanf.c                          0x00000000   Number         0  _chval.o ABSOLUTE
    ../clib/scanf.c                          0x00000000   Number         0  strtol.o ABSOLUTE
    ../clib/scanf.c                          0x00000000   Number         0  _strtoul.o ABSOLUTE
    ../clib/scanf.c                          0x00000000   Number         0  atoi.o ABSOLUTE
    ../fplib/microlib/fpadd.c                0x00000000   Number         0  dadd.o ABSOLUTE
    ../fplib/microlib/fpdiv.c                0x00000000   Number         0  ddiv.o ABSOLUTE
    ../fplib/microlib/fpepilogue.c           0x00000000   Number         0  depilogue.o ABSOLUTE
    ../fplib/microlib/fpfix.c                0x00000000   Number         0  dfixul.o ABSOLUTE
    ../fplib/microlib/fpmul.c                0x00000000   Number         0  dmul.o ABSOLUTE
    ..\..\..\..\Library\Device\Nuvoton\NUC200Series\Source\ARM\startup_NUC200Series.s 0x00000000   Number         0  startup_nuc200series.o ABSOLUTE
    ..\..\..\..\Library\Device\Nuvoton\NUC200Series\Source\system_NUC200Series.c 0x00000000   Number         0  system_nuc200series.o ABSOLUTE
    ..\..\..\..\Library\StdDriver\src\adc.c  0x00000000   Number         0  adc.o ABSOLUTE
    ..\..\..\..\Library\StdDriver\src\clk.c  0x00000000   Number         0  clk.o ABSOLUTE
    ..\..\..\..\Library\StdDriver\src\retarget.c 0x00000000   Number         0  retarget.o ABSOLUTE
    ..\..\..\..\Library\StdDriver\src\sys.c  0x00000000   Number         0  sys.o ABSOLUTE
    ..\..\..\..\Library\StdDriver\src\uart.c 0x00000000   Number         0  uart.o ABSOLUTE
    ..\..\..\..\bsp\chip_uip_interrupt.c     0x00000000   Number         0  chip_uip_interrupt.o ABSOLUTE
    ..\..\..\..\bsp\hardware_init.c          0x00000000   Number         0  hardware_init.o ABSOLUTE
    ..\..\..\..\uipkernel\uip_kernel_common.c 0x00000000   Number         0  uip_kernel_common.o ABSOLUTE
    ..\..\..\..\uipkernel\uip_kernel_event.c 0x00000000   Number         0  uip_kernel_event.o ABSOLUTE
    ..\..\..\..\uipkernel\uip_kernel_isr_cm.s 0x00000000   Number         0  uip_kernel_isr_cm.o ABSOLUTE
    ..\..\..\..\uipkernel\uip_kernel_isr_engine.c 0x00000000   Number         0  uip_kernel_isr_engine.o ABSOLUTE
    ..\..\..\..\uipkernel\uip_kernel_message.c 0x00000000   Number         0  uip_kernel_message.o ABSOLUTE
    ..\..\..\..\uipkernel\uip_kernel_resource.c 0x00000000   Number         0  uip_kernel_resource.o ABSOLUTE
    ..\..\..\..\uipkernel\uip_kernel_scheduler.c 0x00000000   Number         0  uip_kernel_scheduler.o ABSOLUTE
    ..\..\..\..\uipkernel\uip_kernel_task.c  0x00000000   Number         0  uip_kernel_task.o ABSOLUTE
    ..\..\..\..\uipkernel\uip_kernel_time.c  0x00000000   Number         0  uip_kernel_time.o ABSOLUTE
    ..\\..\\..\\..\\Library\\Device\\Nuvoton\\NUC200Series\\Source\\system_NUC200Series.c 0x00000000   Number         0  system_nuc200series.o ABSOLUTE
    ..\\..\\..\\..\\Library\\StdDriver\\src\\adc.c 0x00000000   Number         0  adc.o ABSOLUTE
    ..\\..\\..\\..\\Library\\StdDriver\\src\\clk.c 0x00000000   Number         0  clk.o ABSOLUTE
    ..\\..\\..\\..\\Library\\StdDriver\\src\\retarget.c 0x00000000   Number         0  retarget.o ABSOLUTE
    ..\\..\\..\\..\\Library\\StdDriver\\src\\sys.c 0x00000000   Number         0  sys.o ABSOLUTE
    ..\\..\\..\\..\\Library\\StdDriver\\src\\uart.c 0x00000000   Number         0  uart.o ABSOLUTE
    ..\\..\\..\\..\\bsp\\hardware_init.c     0x00000000   Number         0  hardware_init.o ABSOLUTE
    app\\demo.c                              0x00000000   Number         0  demo.o ABSOLUTE
    app\\init.c                              0x00000000   Number         0  init.o ABSOLUTE
    app\app_cfg.c                            0x00000000   Number         0  app_cfg.o ABSOLUTE
    app\app_int_cfg.c                        0x00000000   Number         0  app_int_cfg.o ABSOLUTE
    app\demo.c                               0x00000000   Number         0  demo.o ABSOLUTE
    app\hook.c                               0x00000000   Number         0  hook.o ABSOLUTE
    app\init.c                               0x00000000   Number         0  init.o ABSOLUTE
    cdrcmple.s                               0x00000000   Number         0  cdrcmple.o ABSOLUTE
    handlers.s                               0x00000000   Number         0  handlers.o ABSOLUTE
    init.s                                   0x00000000   Number         0  init.o ABSOLUTE
    .ARM.Collect$$$$00000000                 0x000000c0   Section        0  entry.o(.ARM.Collect$$$$00000000)
    .ARM.Collect$$$$00000001                 0x000000c0   Section        4  entry2.o(.ARM.Collect$$$$00000001)
    .ARM.Collect$$$$00000004                 0x000000c4   Section        4  entry5.o(.ARM.Collect$$$$00000004)
    .ARM.Collect$$$$00000008                 0x000000c8   Section        0  entry7b.o(.ARM.Collect$$$$00000008)
    .ARM.Collect$$$$0000000A                 0x000000c8   Section        0  entry8b.o(.ARM.Collect$$$$0000000A)
    .ARM.Collect$$$$0000000B                 0x000000c8   Section        8  entry9a.o(.ARM.Collect$$$$0000000B)
    .ARM.Collect$$$$0000000D                 0x000000d0   Section        0  entry10a.o(.ARM.Collect$$$$0000000D)
    .ARM.Collect$$$$0000000F                 0x000000d0   Section        0  entry11a.o(.ARM.Collect$$$$0000000F)
    .ARM.Collect$$$$00002712                 0x000000d0   Section        4  entry2.o(.ARM.Collect$$$$00002712)
    __lit__00000000                          0x000000d0   Data           4  entry2.o(.ARM.Collect$$$$00002712)
    .emb_text                                0x000000d4   Section       28  retarget.o(.emb_text)
    .text                                    0x000000f0   Section       76  startup_nuc200series.o(.text)
    Default_Handler                          0x0000011b   Thumb Code     2  startup_nuc200series.o(.text)
    .text                                    0x0000013c   Section        0  uidiv.o(.text)
    .text                                    0x00000168   Section        0  uldiv.o(.text)
    .text                                    0x000001c8   Section        0  atoi.o(.text)
    .text                                    0x000001e2   Section        0  llshl.o(.text)
    .text                                    0x00000202   Section        0  llushr.o(.text)
    .text                                    0x00000224   Section        0  strtol.o(.text)
    .text                                    0x00000294   Section       36  init.o(.text)
    .text                                    0x000002b8   Section        0  ctype_o.o(.text)
    .text                                    0x000002c0   Section        0  _strtoul.o(.text)
    .text                                    0x00000366   Section        0  _chval.o(.text)
    CODE                                     0x00000384   Section       88  uip_kernel_isr_cm.o(CODE)
    i.ACMP_IRQHandler                        0x000003dc   Section        0  chip_uip_interrupt.o(i.ACMP_IRQHandler)
    i.ADC_DisableInt                         0x000003f0   Section        0  adc.o(i.ADC_DisableInt)
    i.ADC_EnableInt                          0x00000414   Section        0  adc.o(i.ADC_EnableInt)
    i.ADC_IRQHandler                         0x00000438   Section        0  chip_uip_interrupt.o(i.ADC_IRQHandler)
    i.ADC_IRQHandler_Process                 0x0000044c   Section        0  init.o(i.ADC_IRQHandler_Process)
    i.ADC_Open                               0x0000046c   Section        0  adc.o(i.ADC_Open)
    i.AppIdleTask                            0x0000048c   Section        0  demo.o(i.AppIdleTask)
    i.BOD_IRQHandler                         0x000004ac   Section        0  chip_uip_interrupt.o(i.BOD_IRQHandler)
    i.CAN0_IRQHandler                        0x000004c0   Section        0  chip_uip_interrupt.o(i.CAN0_IRQHandler)
    i.CAN1_IRQHandler                        0x000004d4   Section        0  chip_uip_interrupt.o(i.CAN1_IRQHandler)
    i.CLK_EnableModuleClock                  0x000004e8   Section        0  clk.o(i.CLK_EnableModuleClock)
    i.CLK_EnablePLL                          0x00000518   Section        0  clk.o(i.CLK_EnablePLL)
    i.CLK_EnableXtalRC                       0x000006b0   Section        0  clk.o(i.CLK_EnableXtalRC)
    i.CLK_GetPLLClockFreq                    0x000006c0   Section        0  uart.o(i.CLK_GetPLLClockFreq)
    CLK_GetPLLClockFreq                      0x000006c1   Thumb Code    70  uart.o(i.CLK_GetPLLClockFreq)
    i.CLK_SetCoreClock                       0x00000718   Section        0  clk.o(i.CLK_SetCoreClock)
    i.CLK_SetHCLK                            0x00000790   Section        0  clk.o(i.CLK_SetHCLK)
    i.CLK_SetModuleClock                     0x000007d8   Section        0  clk.o(i.CLK_SetModuleClock)
    i.CLK_WaitClockReady                     0x000008a4   Section        0  clk.o(i.CLK_WaitClockReady)
    i.Chip_NUC200_ADC_ISR_Handler_Callback   0x000008d0   Section        0  app_int_cfg.o(i.Chip_NUC200_ADC_ISR_Handler_Callback)
    i.EINT0_IRQHandler                       0x000008d4   Section        0  chip_uip_interrupt.o(i.EINT0_IRQHandler)
    i.EINT1_IRQHandler                       0x000008e8   Section        0  chip_uip_interrupt.o(i.EINT1_IRQHandler)
    i.GPAB_IRQHandler                        0x000008fc   Section        0  chip_uip_interrupt.o(i.GPAB_IRQHandler)
    i.GPCDEF_IRQHandler                      0x00000910   Section        0  chip_uip_interrupt.o(i.GPCDEF_IRQHandler)
    i.GetAVDDCodeByADC                       0x00000924   Section        0  init.o(i.GetAVDDCodeByADC)
    i.GetAVDDVoltage                         0x000009b4   Section        0  init.o(i.GetAVDDVoltage)
    i.Hard_Fault_Handler                     0x000009cc   Section        0  retarget.o(i.Hard_Fault_Handler)
    __tagsym$$used                           0x000009cd   Number         0  retarget.o(i.Hard_Fault_Handler)
    i.Hardware_Init                          0x000009f4   Section        0  hardware_init.o(i.Hardware_Init)
    i.I2C0_IRQHandler                        0x000009f8   Section        0  chip_uip_interrupt.o(i.I2C0_IRQHandler)
    i.I2C1_IRQHandler                        0x00000a0c   Section        0  chip_uip_interrupt.o(i.I2C1_IRQHandler)
    i.I2S_IRQHandler                         0x00000a20   Section        0  chip_uip_interrupt.o(i.I2S_IRQHandler)
    i.InterruptHandler                       0x00000a34   Section        0  chip_uip_interrupt.o(i.InterruptHandler)
    i.Kernel_System_Tick_Init                0x00000a84   Section        0  hardware_init.o(i.Kernel_System_Tick_Init)
    i.PDMA_IRQHandler                        0x00000ac4   Section        0  chip_uip_interrupt.o(i.PDMA_IRQHandler)
    i.PS2_IRQHandler                         0x00000ad8   Section        0  chip_uip_interrupt.o(i.PS2_IRQHandler)
    i.PWMA_IRQHandler                        0x00000aec   Section        0  chip_uip_interrupt.o(i.PWMA_IRQHandler)
    i.PWMB_IRQHandler                        0x00000b00   Section        0  chip_uip_interrupt.o(i.PWMB_IRQHandler)
    i.PWRWU_IRQHandler                       0x00000b14   Section        0  chip_uip_interrupt.o(i.PWRWU_IRQHandler)
    i.RTC_IRQHandler                         0x00000b28   Section        0  chip_uip_interrupt.o(i.RTC_IRQHandler)
    i.SC012_IRQHandler                       0x00000b3c   Section        0  chip_uip_interrupt.o(i.SC012_IRQHandler)
    i.SPI0_IRQHandler                        0x00000b50   Section        0  chip_uip_interrupt.o(i.SPI0_IRQHandler)
    i.SPI1_IRQHandler                        0x00000b64   Section        0  chip_uip_interrupt.o(i.SPI1_IRQHandler)
    i.SPI2_IRQHandler                        0x00000b78   Section        0  chip_uip_interrupt.o(i.SPI2_IRQHandler)
    i.SPI3_IRQHandler                        0x00000b8c   Section        0  chip_uip_interrupt.o(i.SPI3_IRQHandler)
    i.SYS_Init                               0x00000ba0   Section        0  init.o(i.SYS_Init)
    i.SYS_ResetModule                        0x00000c3c   Section        0  sys.o(i.SYS_ResetModule)
    i.SendChar_ToUART                        0x00000c58   Section        0  retarget.o(i.SendChar_ToUART)
    i.StartOS                                0x00000c78   Section        0  uip_kernel_common.o(i.StartOS)
    i.SystemCoreClockUpdate                  0x00000ca8   Section        0  system_nuc200series.o(i.SystemCoreClockUpdate)
    i.SystemInit                             0x00000d38   Section        0  system_nuc200series.o(i.SystemInit)
    i.TASK_0                                 0x00000d3a   Section        0  demo.o(i.TASK_0)
    i.TASK_1                                 0x00000d54   Section        0  demo.o(i.TASK_1)
    i.TASK_2                                 0x00000d6c   Section        0  demo.o(i.TASK_2)
    i.TASK_3                                 0x00000d9c   Section        0  demo.o(i.TASK_3)
    i.TASK_4                                 0x00000dc4   Section        0  demo.o(i.TASK_4)
    i.TMR0_IRQHandler                        0x00000df8   Section        0  chip_uip_interrupt.o(i.TMR0_IRQHandler)
    i.TMR1_IRQHandler                        0x00000e0c   Section        0  chip_uip_interrupt.o(i.TMR1_IRQHandler)
    i.TMR2_IRQHandler                        0x00000e20   Section        0  chip_uip_interrupt.o(i.TMR2_IRQHandler)
    i.TMR3_IRQHandler                        0x00000e34   Section        0  chip_uip_interrupt.o(i.TMR3_IRQHandler)
    i.UART02_IRQHandler                      0x00000e48   Section        0  chip_uip_interrupt.o(i.UART02_IRQHandler)
    i.UART0_Init                             0x00000e5c   Section        0  init.o(i.UART0_Init)
    i.UART1_IRQHandler                       0x00000e78   Section        0  chip_uip_interrupt.o(i.UART1_IRQHandler)
    i.UART_Open                              0x00000e8c   Section        0  uart.o(i.UART_Open)
    i.UIP_ActivateTask                       0x00000f14   Section        0  uip_kernel_task.o(i.UIP_ActivateTask)
    i.UIP_ClearEvent                         0x00000fec   Section        0  uip_kernel_event.o(i.UIP_ClearEvent)
    i.UIP_GetResource                        0x00001038   Section        0  uip_kernel_resource.o(i.UIP_GetResource)
    i.UIP_ReceiveMessage                     0x000010dc   Section        0  uip_kernel_message.o(i.UIP_ReceiveMessage)
    i.UIP_ReleaseResource                    0x0000118c   Section        0  uip_kernel_resource.o(i.UIP_ReleaseResource)
    i.UIP_SendMessage                        0x0000128c   Section        0  uip_kernel_message.o(i.UIP_SendMessage)
    i.UIP_SetEvent                           0x00001368   Section        0  uip_kernel_event.o(i.UIP_SetEvent)
    i.UIP_TerminateTask                      0x00001464   Section        0  uip_kernel_task.o(i.UIP_TerminateTask)
    i.UIP_WaitEvent                          0x0000155c   Section        0  uip_kernel_event.o(i.UIP_WaitEvent)
    i.USBD_IRQHandler                        0x000015e0   Section        0  chip_uip_interrupt.o(i.USBD_IRQHandler)
    i.WDT_IRQHandler                         0x000015f4   Section        0  chip_uip_interrupt.o(i.WDT_IRQHandler)
    i.__0printf$5                            0x00001608   Section        0  printf5.o(i.__0printf$5)
    i.__0sprintf$5                           0x00001628   Section        0  printf5.o(i.__0sprintf$5)
    i.__aeabi_errno_addr                     0x00001650   Section        0  errno.o(i.__aeabi_errno_addr)
    i.__scatterload_copy                     0x00001658   Section       14  handlers.o(i.__scatterload_copy)
    i.__scatterload_null                     0x00001666   Section        2  handlers.o(i.__scatterload_null)
    i.__scatterload_zeroinit                 0x00001668   Section       14  handlers.o(i.__scatterload_zeroinit)
    i._printf_core                           0x00001678   Section        0  printf5.o(i._printf_core)
    _printf_core                             0x00001679   Thumb Code   688  printf5.o(i._printf_core)
    i._sputc                                 0x00001954   Section        0  printf5.o(i._sputc)
    _sputc                                   0x00001955   Thumb Code    10  printf5.o(i._sputc)
    i.fputc                                  0x0000195e   Section        0  retarget.o(i.fputc)
    i.main                                   0x0000196c   Section        0  demo.o(i.main)
    i.pre_main_init                          0x00001988   Section        0  init.o(i.pre_main_init)
    i.stackDump                              0x000019b0   Section        0  retarget.o(i.stackDump)
    stackDump                                0x000019b1   Thumb Code    70  retarget.o(i.stackDump)
    i.uipAlarmInitialize                     0x00001a58   Section        0  uip_kernel_common.o(i.uipAlarmInitialize)
    i.uipAppInitialize                       0x00001a7c   Section        0  demo.o(i.uipAppInitialize)
    i.uipClearPrioGrpAndArrayBit             0x00001adc   Section        0  uip_kernel_scheduler.o(i.uipClearPrioGrpAndArrayBit)
    i.uipGetNextPriority                     0x00001b1c   Section        0  uip_kernel_scheduler.o(i.uipGetNextPriority)
    i.uipGetNextTask                         0x00001b64   Section        0  uip_kernel_scheduler.o(i.uipGetNextTask)
    i.uipInterruptHandlingCallback           0x00001bd0   Section        0  chip_uip_interrupt.o(i.uipInterruptHandlingCallback)
    i.uipInterruptServiceEngine              0x00001be8   Section        0  uip_kernel_isr_engine.o(i.uipInterruptServiceEngine)
    i.uipKernelInitialize                    0x00001c94   Section        0  uip_kernel_common.o(i.uipKernelInitialize)
    i.uipMsgInitialize                       0x00001d54   Section        0  uip_kernel_common.o(i.uipMsgInitialize)
    i.uipPreContexSwitch                     0x00001d88   Section        0  uip_kernel_scheduler.o(i.uipPreContexSwitch)
    i.uipResInitialize                       0x00001db0   Section        0  uip_kernel_common.o(i.uipResInitialize)
    i.uipResetPrioGrpAndArrayBit             0x00001df8   Section        0  uip_kernel_scheduler.o(i.uipResetPrioGrpAndArrayBit)
    i.uipTaskInitialize                      0x00001e20   Section        0  uip_kernel_common.o(i.uipTaskInitialize)
    i.uipTaskStackInit                       0x00001efc   Section        0  uip_kernel_common.o(i.uipTaskStackInit)
    .constdata                               0x00001f44   Section       56  clk.o(.constdata)
    .constdata                               0x00001f7c   Section       48  uart.o(.constdata)
    .constdata                               0x00001fac   Section      129  ctype_o.o(.constdata)
    .constdata                               0x00002030   Section        4  ctype_o.o(.constdata)
    table                                    0x00002030   Data           4  ctype_o.o(.constdata)
    .data                                    0x20000000   Section       44  system_nuc200series.o(.data)
    .data                                    0x2000002c   Section       24  app_cfg.o(.data)
    .data                                    0x20000044   Section       24  app_cfg.o(.data)
    .data                                    0x2000005c   Section       48  app_cfg.o(.data)
    .data                                    0x2000008c   Section        1  app_cfg.o(.data)
    .data                                    0x20000090   Section       20  app_cfg.o(.data)
    .data                                    0x200000a4   Section        1  app_cfg.o(.data)
    .data                                    0x200000a8   Section       36  app_cfg.o(.data)
    .data                                    0x200000cc   Section        1  app_cfg.o(.data)
    .data                                    0x200000d0   Section      288  app_cfg.o(.data)
    .data                                    0x200001f0   Section        1  app_cfg.o(.data)
    .data                                    0x200001f1   Section        4  app_cfg.o(.data)
    .data                                    0x200001f8   Section       32  app_int_cfg.o(.data)
    .data                                    0x20000218   Section        1  app_int_cfg.o(.data)
    .data                                    0x20000219   Section        4  app_int_cfg.o(.data)
    .data                                    0x20000220   Section        4  retarget.o(.data)
    .data                                    0x20000224   Section       32  uip_kernel_common.o(.data)
    .data                                    0x20000244   Section        1  uip_kernel_common.o(.data)
    .data                                    0x20000248   Section      272  uip_kernel_scheduler.o(.data)
    .data                                    0x20000358   Section        1  uip_kernel_scheduler.o(.data)
    .data                                    0x2000035c   Section        4  uip_kernel_scheduler.o(.data)
    .data                                    0x20000360   Section        1  uip_kernel_scheduler.o(.data)
    .data                                    0x20000364   Section        4  uip_kernel_scheduler.o(.data)
    .data                                    0x20000368   Section        4  errno.o(.data)
    _errno                                   0x20000368   Data           4  errno.o(.data)
    .bss                                     0x2000036c   Section      288  app_cfg.o(.bss)
    .bss                                     0x2000048c   Section      288  app_cfg.o(.bss)
    .bss                                     0x200005ac   Section      288  app_cfg.o(.bss)
    .bss                                     0x200006cc   Section      288  app_cfg.o(.bss)
    .bss                                     0x200007ec   Section      288  app_cfg.o(.bss)
    .bss                                     0x2000090c   Section      288  app_cfg.o(.bss)
    .bss                                     0x20000a2c   Section      104  uip_kernel_common.o(.bss)
    STACK                                    0x20000a98   Section     1024  startup_nuc200series.o(STACK)

    Global Symbols

    Symbol Name                              Value     Ov Type        Size  Object(Section)

    BuildAttributes$$THM_ISAv3M$S$PE$A:L22$X:L11$S22$IEEE1$IW$USESV6$~STKCKD$USESV7$~SHL$OSPACE$ROPI$EBA8$MICROLIB$REQ8$PRES8$EABIv2 0x00000000   Number         0  anon$$obj.o ABSOLUTE
    __ARM_use_no_argv                        0x00000000   Number         0  demo.o ABSOLUTE
    __Vectors                                0x00000000   Data           4  startup_nuc200series.o(RESET)
    _printf_a                                0x00000000   Number         0  stubs.o ABSOLUTE
    _printf_c                                0x00000000   Number         0  stubs.o ABSOLUTE
    _printf_charcount                        0x00000000   Number         0  stubs.o ABSOLUTE
    _printf_d                                0x00000000   Number         0  stubs.o ABSOLUTE
    _printf_e                                0x00000000   Number         0  stubs.o ABSOLUTE
    _printf_f                                0x00000000   Number         0  stubs.o ABSOLUTE
    _printf_flags                            0x00000000   Number         0  stubs.o ABSOLUTE
    _printf_fp_dec                           0x00000000   Number         0  stubs.o ABSOLUTE
    _printf_fp_hex                           0x00000000   Number         0  stubs.o ABSOLUTE
    _printf_g                                0x00000000   Number         0  stubs.o ABSOLUTE
    _printf_i                                0x00000000   Number         0  stubs.o ABSOLUTE
    _printf_int_dec                          0x00000000   Number         0  stubs.o ABSOLUTE
    _printf_l                                0x00000000   Number         0  stubs.o ABSOLUTE
    _printf_lc                               0x00000000   Number         0  stubs.o ABSOLUTE
    _printf_ll                               0x00000000   Number         0  stubs.o ABSOLUTE
    _printf_lld                              0x00000000   Number         0  stubs.o ABSOLUTE
    _printf_lli                              0x00000000   Number         0  stubs.o ABSOLUTE
    _printf_llo                              0x00000000   Number         0  stubs.o ABSOLUTE
    _printf_llu                              0x00000000   Number         0  stubs.o ABSOLUTE
    _printf_llx                              0x00000000   Number         0  stubs.o ABSOLUTE
    _printf_longlong_dec                     0x00000000   Number         0  stubs.o ABSOLUTE
    _printf_longlong_hex                     0x00000000   Number         0  stubs.o ABSOLUTE
    _printf_longlong_oct                     0x00000000   Number         0  stubs.o ABSOLUTE
    _printf_ls                               0x00000000   Number         0  stubs.o ABSOLUTE
    _printf_mbtowc                           0x00000000   Number         0  stubs.o ABSOLUTE
    _printf_n                                0x00000000   Number         0  stubs.o ABSOLUTE
    _printf_o                                0x00000000   Number         0  stubs.o ABSOLUTE
    _printf_p                                0x00000000   Number         0  stubs.o ABSOLUTE
    _printf_percent                          0x00000000   Number         0  stubs.o ABSOLUTE
    _printf_pre_padding                      0x00000000   Number         0  stubs.o ABSOLUTE
    _printf_return_value                     0x00000000   Number         0  stubs.o ABSOLUTE
    _printf_s                                0x00000000   Number         0  stubs.o ABSOLUTE
    _printf_sizespec                         0x00000000   Number         0  stubs.o ABSOLUTE
    _printf_str                              0x00000000   Number         0  stubs.o ABSOLUTE
    _printf_truncate_signed                  0x00000000   Number         0  stubs.o ABSOLUTE
    _printf_truncate_unsigned                0x00000000   Number         0  stubs.o ABSOLUTE
    _printf_u                                0x00000000   Number         0  stubs.o ABSOLUTE
    _printf_wc                               0x00000000   Number         0  stubs.o ABSOLUTE
    _printf_wctomb                           0x00000000   Number         0  stubs.o ABSOLUTE
    _printf_widthprec                        0x00000000   Number         0  stubs.o ABSOLUTE
    _printf_x                                0x00000000   Number         0  stubs.o ABSOLUTE
    __cpp_initialize__aeabi_                  - Undefined Weak Reference
    __cxa_finalize                            - Undefined Weak Reference
    __decompress                              - Undefined Weak Reference
    _clock_init                               - Undefined Weak Reference
    _microlib_exit                            - Undefined Weak Reference
    __main                                   0x000000c1   Thumb Code     0  entry.o(.ARM.Collect$$$$00000000)
    _main_stk                                0x000000c1   Thumb Code     0  entry2.o(.ARM.Collect$$$$00000001)
    _main_scatterload                        0x000000c5   Thumb Code     0  entry5.o(.ARM.Collect$$$$00000004)
    __main_after_scatterload                 0x000000c9   Thumb Code     0  entry5.o(.ARM.Collect$$$$00000004)
    _main_clock                              0x000000c9   Thumb Code     0  entry7b.o(.ARM.Collect$$$$00000008)
    _main_cpp_init                           0x000000c9   Thumb Code     0  entry8b.o(.ARM.Collect$$$$0000000A)
    _main_init                               0x000000c9   Thumb Code     0  entry9a.o(.ARM.Collect$$$$0000000B)
    __rt_final_cpp                           0x000000d1   Thumb Code     0  entry10a.o(.ARM.Collect$$$$0000000D)
    __rt_final_exit                          0x000000d1   Thumb Code     0  entry11a.o(.ARM.Collect$$$$0000000F)
    HardFault_Handler                        0x000000d5   Thumb Code    24  retarget.o(.emb_text)
    Reset_Handler                            0x000000f1   Thumb Code    32  startup_nuc200series.o(.text)
    NMI_Handler                              0x00000111   Thumb Code     2  startup_nuc200series.o(.text)
    SVC_Handler                              0x00000115   Thumb Code     2  startup_nuc200series.o(.text)
    PendSV_Handler                           0x00000117   Thumb Code     2  startup_nuc200series.o(.text)
    SysTick_Handler                          0x00000119   Thumb Code     2  startup_nuc200series.o(.text)
    __aeabi_uidiv                            0x0000013d   Thumb Code     0  uidiv.o(.text)
    __aeabi_uidivmod                         0x0000013d   Thumb Code    44  uidiv.o(.text)
    __aeabi_uldivmod                         0x00000169   Thumb Code    96  uldiv.o(.text)
    atoi                                     0x000001c9   Thumb Code    26  atoi.o(.text)
    __aeabi_llsl                             0x000001e3   Thumb Code    32  llshl.o(.text)
    _ll_shift_l                              0x000001e3   Thumb Code     0  llshl.o(.text)
    __aeabi_llsr                             0x00000203   Thumb Code    34  llushr.o(.text)
    _ll_ushift_r                             0x00000203   Thumb Code     0  llushr.o(.text)
    strtol                                   0x00000225   Thumb Code   108  strtol.o(.text)
    __scatterload                            0x00000295   Thumb Code    28  init.o(.text)
    __scatterload_rt2                        0x00000295   Thumb Code     0  init.o(.text)
    __rt_ctype_table                         0x000002b9   Thumb Code     4  ctype_o.o(.text)
    _strtoul                                 0x000002c1   Thumb Code   166  _strtoul.o(.text)
    _chval                                   0x00000367   Thumb Code    30  _chval.o(.text)
    uipDisableAllInterrupts                  0x00000385   Thumb Code     0  uip_kernel_isr_cm.o(CODE)
    uipIntMaskStateRestore                   0x0000038d   Thumb Code     0  uip_kernel_isr_cm.o(CODE)
    uipPendSVHandler                         0x00000393   Thumb Code     0  uip_kernel_isr_cm.o(CODE)
    ACMP_IRQHandler                          0x000003dd   Thumb Code    14  chip_uip_interrupt.o(i.ACMP_IRQHandler)
    ADC_DisableInt                           0x000003f1   Thumb Code    36  adc.o(i.ADC_DisableInt)
    ADC_EnableInt                            0x00000415   Thumb Code    36  adc.o(i.ADC_EnableInt)
    ADC_IRQHandler                           0x00000439   Thumb Code    14  chip_uip_interrupt.o(i.ADC_IRQHandler)
    ADC_IRQHandler_Process                   0x0000044d   Thumb Code    26  init.o(i.ADC_IRQHandler_Process)
    ADC_Open                                 0x0000046d   Thumb Code    26  adc.o(i.ADC_Open)
    AppIdleTask                              0x0000048d   Thumb Code    28  demo.o(i.AppIdleTask)
    BOD_IRQHandler                           0x000004ad   Thumb Code    14  chip_uip_interrupt.o(i.BOD_IRQHandler)
    CAN0_IRQHandler                          0x000004c1   Thumb Code    14  chip_uip_interrupt.o(i.CAN0_IRQHandler)
    CAN1_IRQHandler                          0x000004d5   Thumb Code    14  chip_uip_interrupt.o(i.CAN1_IRQHandler)
    CLK_EnableModuleClock                    0x000004e9   Thumb Code    40  clk.o(i.CLK_EnableModuleClock)
    CLK_EnablePLL                            0x00000519   Thumb Code   348  clk.o(i.CLK_EnablePLL)
    CLK_EnableXtalRC                         0x000006b1   Thumb Code    10  clk.o(i.CLK_EnableXtalRC)
    CLK_SetCoreClock                         0x00000719   Thumb Code   112  clk.o(i.CLK_SetCoreClock)
    CLK_SetHCLK                              0x00000791   Thumb Code    66  clk.o(i.CLK_SetHCLK)
    CLK_SetModuleClock                       0x000007d9   Thumb Code   180  clk.o(i.CLK_SetModuleClock)
    CLK_WaitClockReady                       0x000008a5   Thumb Code    34  clk.o(i.CLK_WaitClockReady)
    Chip_NUC200_ADC_ISR_Handler_Callback     0x000008d1   Thumb Code     4  app_int_cfg.o(i.Chip_NUC200_ADC_ISR_Handler_Callback)
    EINT0_IRQHandler                         0x000008d5   Thumb Code    14  chip_uip_interrupt.o(i.EINT0_IRQHandler)
    EINT1_IRQHandler                         0x000008e9   Thumb Code    14  chip_uip_interrupt.o(i.EINT1_IRQHandler)
    GPAB_IRQHandler                          0x000008fd   Thumb Code    14  chip_uip_interrupt.o(i.GPAB_IRQHandler)
    GPCDEF_IRQHandler                        0x00000911   Thumb Code    14  chip_uip_interrupt.o(i.GPCDEF_IRQHandler)
    GetAVDDCodeByADC                         0x00000925   Thumb Code   128  init.o(i.GetAVDDCodeByADC)
    GetAVDDVoltage                           0x000009b5   Thumb Code    22  init.o(i.GetAVDDVoltage)
    Hard_Fault_Handler                       0x000009cd   Thumb Code    16  retarget.o(i.Hard_Fault_Handler)
    Hardware_Init                            0x000009f5   Thumb Code     2  hardware_init.o(i.Hardware_Init)
    I2C0_IRQHandler                          0x000009f9   Thumb Code    14  chip_uip_interrupt.o(i.I2C0_IRQHandler)
    I2C1_IRQHandler                          0x00000a0d   Thumb Code    14  chip_uip_interrupt.o(i.I2C1_IRQHandler)
    I2S_IRQHandler                           0x00000a21   Thumb Code    14  chip_uip_interrupt.o(i.I2S_IRQHandler)
    InterruptHandler                         0x00000a35   Thumb Code    66  chip_uip_interrupt.o(i.InterruptHandler)
    Kernel_System_Tick_Init                  0x00000a85   Thumb Code    48  hardware_init.o(i.Kernel_System_Tick_Init)
    PDMA_IRQHandler                          0x00000ac5   Thumb Code    14  chip_uip_interrupt.o(i.PDMA_IRQHandler)
    PS2_IRQHandler                           0x00000ad9   Thumb Code    14  chip_uip_interrupt.o(i.PS2_IRQHandler)
    PWMA_IRQHandler                          0x00000aed   Thumb Code    14  chip_uip_interrupt.o(i.PWMA_IRQHandler)
    PWMB_IRQHandler                          0x00000b01   Thumb Code    14  chip_uip_interrupt.o(i.PWMB_IRQHandler)
    PWRWU_IRQHandler                         0x00000b15   Thumb Code    14  chip_uip_interrupt.o(i.PWRWU_IRQHandler)
    RTC_IRQHandler                           0x00000b29   Thumb Code    14  chip_uip_interrupt.o(i.RTC_IRQHandler)
    SC012_IRQHandler                         0x00000b3d   Thumb Code    14  chip_uip_interrupt.o(i.SC012_IRQHandler)
    SPI0_IRQHandler                          0x00000b51   Thumb Code    14  chip_uip_interrupt.o(i.SPI0_IRQHandler)
    SPI1_IRQHandler                          0x00000b65   Thumb Code    14  chip_uip_interrupt.o(i.SPI1_IRQHandler)
    SPI2_IRQHandler                          0x00000b79   Thumb Code    14  chip_uip_interrupt.o(i.SPI2_IRQHandler)
    SPI3_IRQHandler                          0x00000b8d   Thumb Code    14  chip_uip_interrupt.o(i.SPI3_IRQHandler)
    SYS_Init                                 0x00000ba1   Thumb Code   136  init.o(i.SYS_Init)
    SYS_ResetModule                          0x00000c3d   Thumb Code    26  sys.o(i.SYS_ResetModule)
    SendChar_ToUART                          0x00000c59   Thumb Code    26  retarget.o(i.SendChar_ToUART)
    StartOS                                  0x00000c79   Thumb Code    38  uip_kernel_common.o(i.StartOS)
    SystemCoreClockUpdate                    0x00000ca9   Thumb Code   118  system_nuc200series.o(i.SystemCoreClockUpdate)
    SystemInit                               0x00000d39   Thumb Code     2  system_nuc200series.o(i.SystemInit)
    TASK_0                                   0x00000d3b   Thumb Code    26  demo.o(i.TASK_0)
    TASK_1                                   0x00000d55   Thumb Code    20  demo.o(i.TASK_1)
    TASK_2                                   0x00000d6d   Thumb Code    44  demo.o(i.TASK_2)
    TASK_3                                   0x00000d9d   Thumb Code    36  demo.o(i.TASK_3)
    TASK_4                                   0x00000dc5   Thumb Code    30  demo.o(i.TASK_4)
    TMR0_IRQHandler                          0x00000df9   Thumb Code    14  chip_uip_interrupt.o(i.TMR0_IRQHandler)
    TMR1_IRQHandler                          0x00000e0d   Thumb Code    14  chip_uip_interrupt.o(i.TMR1_IRQHandler)
    TMR2_IRQHandler                          0x00000e21   Thumb Code    14  chip_uip_interrupt.o(i.TMR2_IRQHandler)
    TMR3_IRQHandler                          0x00000e35   Thumb Code    14  chip_uip_interrupt.o(i.TMR3_IRQHandler)
    UART02_IRQHandler                        0x00000e49   Thumb Code    14  chip_uip_interrupt.o(i.UART02_IRQHandler)
    UART0_Init                               0x00000e5d   Thumb Code    20  init.o(i.UART0_Init)
    UART1_IRQHandler                         0x00000e79   Thumb Code    14  chip_uip_interrupt.o(i.UART1_IRQHandler)
    UART_Open                                0x00000e8d   Thumb Code   120  uart.o(i.UART_Open)
    UIP_ActivateTask                         0x00000f15   Thumb Code   174  uip_kernel_task.o(i.UIP_ActivateTask)
    UIP_ClearEvent                           0x00000fed   Thumb Code    64  uip_kernel_event.o(i.UIP_ClearEvent)
    UIP_GetResource                          0x00001039   Thumb Code   130  uip_kernel_resource.o(i.UIP_GetResource)
    UIP_ReceiveMessage                       0x000010dd   Thumb Code   168  uip_kernel_message.o(i.UIP_ReceiveMessage)
    UIP_ReleaseResource                      0x0000118d   Thumb Code   206  uip_kernel_resource.o(i.UIP_ReleaseResource)
    UIP_SendMessage                          0x0000128d   Thumb Code   212  uip_kernel_message.o(i.UIP_SendMessage)
    UIP_SetEvent                             0x00001369   Thumb Code   208  uip_kernel_event.o(i.UIP_SetEvent)
    UIP_TerminateTask                        0x00001465   Thumb Code   206  uip_kernel_task.o(i.UIP_TerminateTask)
    UIP_WaitEvent                            0x0000155d   Thumb Code   116  uip_kernel_event.o(i.UIP_WaitEvent)
    USBD_IRQHandler                          0x000015e1   Thumb Code    14  chip_uip_interrupt.o(i.USBD_IRQHandler)
    WDT_IRQHandler                           0x000015f5   Thumb Code    14  chip_uip_interrupt.o(i.WDT_IRQHandler)
    __0printf$5                              0x00001609   Thumb Code    24  printf5.o(i.__0printf$5)
    __1printf$5                              0x00001609   Thumb Code     0  printf5.o(i.__0printf$5)
    __2printf                                0x00001609   Thumb Code     0  printf5.o(i.__0printf$5)
    __0sprintf$5                             0x00001629   Thumb Code    36  printf5.o(i.__0sprintf$5)
    __1sprintf$5                             0x00001629   Thumb Code     0  printf5.o(i.__0sprintf$5)
    __2sprintf                               0x00001629   Thumb Code     0  printf5.o(i.__0sprintf$5)
    __aeabi_errno_addr                       0x00001651   Thumb Code     4  errno.o(i.__aeabi_errno_addr)
    __rt_errno_addr                          0x00001651   Thumb Code     0  errno.o(i.__aeabi_errno_addr)
    __scatterload_copy                       0x00001659   Thumb Code    14  handlers.o(i.__scatterload_copy)
    __scatterload_null                       0x00001667   Thumb Code     2  handlers.o(i.__scatterload_null)
    __scatterload_zeroinit                   0x00001669   Thumb Code    14  handlers.o(i.__scatterload_zeroinit)
    fputc                                    0x0000195f   Thumb Code    12  retarget.o(i.fputc)
    main                                     0x0000196d   Thumb Code    24  demo.o(i.main)
    pre_main_init                            0x00001989   Thumb Code    34  init.o(i.pre_main_init)
    uipAlarmInitialize                       0x00001a59   Thumb Code    30  uip_kernel_common.o(i.uipAlarmInitialize)
    uipAppInitialize                         0x00001a7d   Thumb Code    60  demo.o(i.uipAppInitialize)
    uipClearPrioGrpAndArrayBit               0x00001add   Thumb Code    60  uip_kernel_scheduler.o(i.uipClearPrioGrpAndArrayBit)
    uipGetNextPriority                       0x00001b1d   Thumb Code    66  uip_kernel_scheduler.o(i.uipGetNextPriority)
    uipGetNextTask                           0x00001b65   Thumb Code    96  uip_kernel_scheduler.o(i.uipGetNextTask)
    uipInterruptHandlingCallback             0x00001bd1   Thumb Code    18  chip_uip_interrupt.o(i.uipInterruptHandlingCallback)
    uipInterruptServiceEngine                0x00001be9   Thumb Code   140  uip_kernel_isr_engine.o(i.uipInterruptServiceEngine)
    uipKernelInitialize                      0x00001c95   Thumb Code   142  uip_kernel_common.o(i.uipKernelInitialize)
    uipMsgInitialize                         0x00001d55   Thumb Code    46  uip_kernel_common.o(i.uipMsgInitialize)
    uipPreContexSwitch                       0x00001d89   Thumb Code    36  uip_kernel_scheduler.o(i.uipPreContexSwitch)
    uipResInitialize                         0x00001db1   Thumb Code    66  uip_kernel_common.o(i.uipResInitialize)
    uipResetPrioGrpAndArrayBit               0x00001df9   Thumb Code    36  uip_kernel_scheduler.o(i.uipResetPrioGrpAndArrayBit)
    uipTaskInitialize                        0x00001e21   Thumb Code   196  uip_kernel_common.o(i.uipTaskInitialize)
    uipTaskStackInit                         0x00001efd   Thumb Code    72  uip_kernel_common.o(i.uipTaskStackInit)
    __ctype_table                            0x00001fac   Data         129  ctype_o.o(.constdata)
    Region$$Table$$Base                      0x00002034   Number         0  anon$$obj.o(Region$$Table)
    Region$$Table$$Limit                     0x00002054   Number         0  anon$$obj.o(Region$$Table)
    SystemCoreClock                          0x20000000   Data           4  system_nuc200series.o(.data)
    CyclesPerUs                              0x20000004   Data           4  system_nuc200series.o(.data)
    PllClock                                 0x20000008   Data           4  system_nuc200series.o(.data)
    gau32ClkSrcTbl                           0x2000000c   Data          32  system_nuc200series.o(.data)
    AppAlarmBase                             0x2000002c   Data          24  app_cfg.o(.data)
    AppCounter                               0x20000044   Data          24  app_cfg.o(.data)
    AppAlarm                                 0x2000005c   Data          48  app_cfg.o(.data)
    AppAlarmNumber                           0x2000008c   Data           1  app_cfg.o(.data)
    AppRes                                   0x20000090   Data          20  app_cfg.o(.data)
    AppResNumber                             0x200000a4   Data           1  app_cfg.o(.data)
    AppMsg                                   0x200000a8   Data          36  app_cfg.o(.data)
    AppMsgNumber                             0x200000cc   Data           1  app_cfg.o(.data)
    AppTask                                  0x200000d0   Data         288  app_cfg.o(.data)
    AppTaskNumber                            0x200001f0   Data           1  app_cfg.o(.data)
    AppMsgBuf                                0x200001f1   Data           4  app_cfg.o(.data)
    UIP_Exc_VectorTable                      0x200001f8   Data          32  app_int_cfg.o(.data)
    AppIntNumber                             0x20000218   Data           1  app_int_cfg.o(.data)
    ChipNUC200ADCIntHandlingData             0x20000219   Data           4  app_int_cfg.o(.data)
    __stdout                                 0x20000220   Data           4  retarget.o(.data)
    uipLowPowerMode                          0x20000224   Data           1  uip_kernel_common.o(.data)
    uipTaskNumber                            0x20000225   Data           1  uip_kernel_common.o(.data)
    uipTaskIDNumber                          0x20000226   Data           1  uip_kernel_common.o(.data)
    uipResNumber                             0x20000227   Data           1  uip_kernel_common.o(.data)
    uipAlarmNumber                           0x20000228   Data           1  uip_kernel_common.o(.data)
    uipAlarmID                               0x20000229   Data           1  uip_kernel_common.o(.data)
    uipMsgNumber                             0x2000022a   Data           1  uip_kernel_common.o(.data)
    uipTCBArray                              0x2000022c   Data           4  uip_kernel_common.o(.data)
    uipRCBArray                              0x20000230   Data           4  uip_kernel_common.o(.data)
    uipACBArray                              0x20000234   Data           4  uip_kernel_common.o(.data)
    uipMCBArray                              0x20000238   Data           4  uip_kernel_common.o(.data)
    uipIntTableID                            0x2000023c   Data           4  uip_kernel_common.o(.data)
    uipInSchedulerLoop                       0x20000240   Data           4  uip_kernel_common.o(.data)
    uipIdleTaskID                            0x20000244   Data           1  uip_kernel_common.o(.data)
    uipCurrentTaskPriority                   0x20000248   Data           1  uip_kernel_scheduler.o(.data)
    uipNextRunningTaskPriority               0x20000249   Data           1  uip_kernel_scheduler.o(.data)
    uipPrioGrpArray                          0x2000024a   Data           2  uip_kernel_scheduler.o(.data)
    uipPrioGroup                             0x2000024c   Data           4  uip_kernel_scheduler.o(.data)
    uipCurrentTaskTCBPtr                     0x20000250   Data           4  uip_kernel_scheduler.o(.data)
    uipNextRunningTaskTCBPtr                 0x20000254   Data           4  uip_kernel_scheduler.o(.data)
    uipByteValue                             0x20000258   Data         256  uip_kernel_scheduler.o(.data)
    uipSchedulerLock                         0x20000358   Data           1  uip_kernel_scheduler.o(.data)
    uipNestedInterrupts                      0x2000035c   Data           4  uip_kernel_scheduler.o(.data)
    uipSystemMode                            0x20000360   Data           1  uip_kernel_scheduler.o(.data)
    uipSystemStackPtr                        0x20000364   Data           4  uip_kernel_scheduler.o(.data)
    Task_0_Stack                             0x2000036c   Data         288  app_cfg.o(.bss)
    Task_1_Stack                             0x2000048c   Data         288  app_cfg.o(.bss)
    Task_2_Stack                             0x200005ac   Data         288  app_cfg.o(.bss)
    Task_3_Stack                             0x200006cc   Data         288  app_cfg.o(.bss)
    Task_4_Stack                             0x200007ec   Data         288  app_cfg.o(.bss)
    Task_App_Idle_Stack                      0x2000090c   Data         288  app_cfg.o(.bss)
    uipPriorityToTaskID                      0x20000a2c   Data          16  uip_kernel_common.o(.bss)
    uipInitTaskStackPtr                      0x20000a3c   Data          64  uip_kernel_common.o(.bss)
    uipSystemCounter                         0x20000a7c   Data          12  uip_kernel_common.o(.bss)
    uipSystemAlarmBase                       0x20000a88   Data          12  uip_kernel_common.o(.bss)
    __initial_sp                             0x20000e98   Data           0  startup_nuc200series.o(STACK)



==============================================================================

Memory Map of the image

  Image Entry point : 0x000000f1

  Load Region LR_1 (Base: 0x00000000, Size: 0x000023c0, Max: 0xffffffff, ABSOLUTE)

    Execution Region ER_RO (Exec base: 0x00000000, Load base: 0x00000000, Size: 0x00002054, Max: 0xffffffff, ABSOLUTE)

    Exec Addr    Load Addr    Size         Type   Attr      Idx    E Section Name        Object

    0x00000000   0x00000000   0x000000c0   Data   RO          114    RESET               startup_nuc200series.o
    0x000000c0   0x000000c0   0x00000000   Code   RO         1493  * .ARM.Collect$$$$00000000  mc_p.l(entry.o)
    0x000000c0   0x000000c0   0x00000004   Code   RO         1761    .ARM.Collect$$$$00000001  mc_p.l(entry2.o)
    0x000000c4   0x000000c4   0x00000004   Code   RO         1764    .ARM.Collect$$$$00000004  mc_p.l(entry5.o)
    0x000000c8   0x000000c8   0x00000000   Code   RO         1766    .ARM.Collect$$$$00000008  mc_p.l(entry7b.o)
    0x000000c8   0x000000c8   0x00000000   Code   RO         1768    .ARM.Collect$$$$0000000A  mc_p.l(entry8b.o)
    0x000000c8   0x000000c8   0x00000008   Code   RO         1769    .ARM.Collect$$$$0000000B  mc_p.l(entry9a.o)
    0x000000d0   0x000000d0   0x00000000   Code   RO         1771    .ARM.Collect$$$$0000000D  mc_p.l(entry10a.o)
    0x000000d0   0x000000d0   0x00000000   Code   RO         1773    .ARM.Collect$$$$0000000F  mc_p.l(entry11a.o)
    0x000000d0   0x000000d0   0x00000004   Code   RO         1762    .ARM.Collect$$$$00002712  mc_p.l(entry2.o)
    0x000000d4   0x000000d4   0x0000001c   Code   RO          399    .emb_text           retarget.o
    0x000000f0   0x000000f0   0x0000004c   Code   RO          115  * .text               startup_nuc200series.o
    0x0000013c   0x0000013c   0x0000002c   Code   RO         1494    .text               mc_p.l(uidiv.o)
    0x00000168   0x00000168   0x00000060   Code   RO         1496    .text               mc_p.l(uldiv.o)
    0x000001c8   0x000001c8   0x0000001a   Code   RO         1759    .text               mc_p.l(atoi.o)
    0x000001e2   0x000001e2   0x00000020   Code   RO         1775    .text               mc_p.l(llshl.o)
    0x00000202   0x00000202   0x00000022   Code   RO         1777    .text               mc_p.l(llushr.o)
    0x00000224   0x00000224   0x00000070   Code   RO         1786    .text               mc_p.l(strtol.o)
    0x00000294   0x00000294   0x00000024   Code   RO         1799    .text               mc_p.l(init.o)
    0x000002b8   0x000002b8   0x00000008   Code   RO         1803    .text               mc_p.l(ctype_o.o)
    0x000002c0   0x000002c0   0x000000a6   Code   RO         1831    .text               mc_p.l(_strtoul.o)
    0x00000366   0x00000366   0x0000001e   Code   RO         1837    .text               mc_p.l(_chval.o)
    0x00000384   0x00000384   0x00000058   Code   RO         1255    CODE                uip_kernel_isr_cm.o
    0x000003dc   0x000003dc   0x00000014   Code   RO          867    i.ACMP_IRQHandler   chip_uip_interrupt.o
    0x000003f0   0x000003f0   0x00000024   Code   RO          821    i.ADC_DisableInt    adc.o
    0x00000414   0x00000414   0x00000024   Code   RO          823    i.ADC_EnableInt     adc.o
    0x00000438   0x00000438   0x00000014   Code   RO          868    i.ADC_IRQHandler    chip_uip_interrupt.o
    0x0000044c   0x0000044c   0x00000020   Code   RO          340    i.ADC_IRQHandler_Process  init.o
    0x0000046c   0x0000046c   0x00000020   Code   RO          824    i.ADC_Open          adc.o
    0x0000048c   0x0000048c   0x00000020   Code   RO          179    i.AppIdleTask       demo.o
    0x000004ac   0x000004ac   0x00000014   Code   RO          869    i.BOD_IRQHandler    chip_uip_interrupt.o
    0x000004c0   0x000004c0   0x00000014   Code   RO          870    i.CAN0_IRQHandler   chip_uip_interrupt.o
    0x000004d4   0x000004d4   0x00000014   Code   RO          871    i.CAN1_IRQHandler   chip_uip_interrupt.o
    0x000004e8   0x000004e8   0x00000030   Code   RO          494    i.CLK_EnableModuleClock  clk.o
    0x00000518   0x00000518   0x00000198   Code   RO          495    i.CLK_EnablePLL     clk.o
    0x000006b0   0x000006b0   0x00000010   Code   RO          497    i.CLK_EnableXtalRC  clk.o
    0x000006c0   0x000006c0   0x00000058   Code   RO          709    i.CLK_GetPLLClockFreq  uart.o
    0x00000718   0x00000718   0x00000078   Code   RO          505    i.CLK_SetCoreClock  clk.o
    0x00000790   0x00000790   0x00000048   Code   RO          506    i.CLK_SetHCLK       clk.o
    0x000007d8   0x000007d8   0x000000cc   Code   RO          507    i.CLK_SetModuleClock  clk.o
    0x000008a4   0x000008a4   0x0000002c   Code   RO          509    i.CLK_WaitClockReady  clk.o
    0x000008d0   0x000008d0   0x00000004   Code   RO          156    i.Chip_NUC200_ADC_ISR_Handler_Callback  app_int_cfg.o
    0x000008d4   0x000008d4   0x00000014   Code   RO          878    i.EINT0_IRQHandler  chip_uip_interrupt.o
    0x000008e8   0x000008e8   0x00000014   Code   RO          879    i.EINT1_IRQHandler  chip_uip_interrupt.o
    0x000008fc   0x000008fc   0x00000014   Code   RO          880    i.GPAB_IRQHandler   chip_uip_interrupt.o
    0x00000910   0x00000910   0x00000014   Code   RO          881    i.GPCDEF_IRQHandler  chip_uip_interrupt.o
    0x00000924   0x00000924   0x00000090   Code   RO          341    i.GetAVDDCodeByADC  init.o
    0x000009b4   0x000009b4   0x00000016   Code   RO          342    i.GetAVDDVoltage    init.o
    0x000009ca   0x000009ca   0x00000002   PAD
    0x000009cc   0x000009cc   0x00000028   Code   RO          401    i.Hard_Fault_Handler  retarget.o
    0x000009f4   0x000009f4   0x00000002   Code   RO         1112    i.Hardware_Init     hardware_init.o
    0x000009f6   0x000009f6   0x00000002   PAD
    0x000009f8   0x000009f8   0x00000014   Code   RO          882    i.I2C0_IRQHandler   chip_uip_interrupt.o
    0x00000a0c   0x00000a0c   0x00000014   Code   RO          883    i.I2C1_IRQHandler   chip_uip_interrupt.o
    0x00000a20   0x00000a20   0x00000014   Code   RO          884    i.I2S_IRQHandler    chip_uip_interrupt.o
    0x00000a34   0x00000a34   0x00000050   Code   RO          885    i.InterruptHandler  chip_uip_interrupt.o
    0x00000a84   0x00000a84   0x00000040   Code   RO         1113    i.Kernel_System_Tick_Init  hardware_init.o
    0x00000ac4   0x00000ac4   0x00000014   Code   RO          886    i.PDMA_IRQHandler   chip_uip_interrupt.o
    0x00000ad8   0x00000ad8   0x00000014   Code   RO          887    i.PS2_IRQHandler    chip_uip_interrupt.o
    0x00000aec   0x00000aec   0x00000014   Code   RO          888    i.PWMA_IRQHandler   chip_uip_interrupt.o
    0x00000b00   0x00000b00   0x00000014   Code   RO          889    i.PWMB_IRQHandler   chip_uip_interrupt.o
    0x00000b14   0x00000b14   0x00000014   Code   RO          890    i.PWRWU_IRQHandler  chip_uip_interrupt.o
    0x00000b28   0x00000b28   0x00000014   Code   RO          891    i.RTC_IRQHandler    chip_uip_interrupt.o
    0x00000b3c   0x00000b3c   0x00000014   Code   RO          892    i.SC012_IRQHandler  chip_uip_interrupt.o
    0x00000b50   0x00000b50   0x00000014   Code   RO          893    i.SPI0_IRQHandler   chip_uip_interrupt.o
    0x00000b64   0x00000b64   0x00000014   Code   RO          894    i.SPI1_IRQHandler   chip_uip_interrupt.o
    0x00000b78   0x00000b78   0x00000014   Code   RO          895    i.SPI2_IRQHandler   chip_uip_interrupt.o
    0x00000b8c   0x00000b8c   0x00000014   Code   RO          896    i.SPI3_IRQHandler   chip_uip_interrupt.o
    0x00000ba0   0x00000ba0   0x0000009c   Code   RO          343    i.SYS_Init          init.o
    0x00000c3c   0x00000c3c   0x0000001a   Code   RO          644    i.SYS_ResetModule   sys.o
    0x00000c56   0x00000c56   0x00000002   PAD
    0x00000c58   0x00000c58   0x00000020   Code   RO          404    i.SendChar_ToUART   retarget.o
    0x00000c78   0x00000c78   0x00000030   Code   RO         1137    i.StartOS           uip_kernel_common.o
    0x00000ca8   0x00000ca8   0x00000090   Code   RO            3    i.SystemCoreClockUpdate  system_nuc200series.o
    0x00000d38   0x00000d38   0x00000002   Code   RO            4    i.SystemInit        system_nuc200series.o
    0x00000d3a   0x00000d3a   0x0000001a   Code   RO          180    i.TASK_0            demo.o
    0x00000d54   0x00000d54   0x00000018   Code   RO          181    i.TASK_1            demo.o
    0x00000d6c   0x00000d6c   0x00000030   Code   RO          182    i.TASK_2            demo.o
    0x00000d9c   0x00000d9c   0x00000028   Code   RO          183    i.TASK_3            demo.o
    0x00000dc4   0x00000dc4   0x00000034   Code   RO          184    i.TASK_4            demo.o
    0x00000df8   0x00000df8   0x00000014   Code   RO          897    i.TMR0_IRQHandler   chip_uip_interrupt.o
    0x00000e0c   0x00000e0c   0x00000014   Code   RO          898    i.TMR1_IRQHandler   chip_uip_interrupt.o
    0x00000e20   0x00000e20   0x00000014   Code   RO          899    i.TMR2_IRQHandler   chip_uip_interrupt.o
    0x00000e34   0x00000e34   0x00000014   Code   RO          900    i.TMR3_IRQHandler   chip_uip_interrupt.o
    0x00000e48   0x00000e48   0x00000014   Code   RO          901    i.UART02_IRQHandler  chip_uip_interrupt.o
    0x00000e5c   0x00000e5c   0x0000001c   Code   RO          344    i.UART0_Init        init.o
    0x00000e78   0x00000e78   0x00000014   Code   RO          902    i.UART1_IRQHandler  chip_uip_interrupt.o
    0x00000e8c   0x00000e8c   0x00000088   Code   RO          716    i.UART_Open         uart.o
    0x00000f14   0x00000f14   0x000000d8   Code   RO         1391    i.UIP_ActivateTask  uip_kernel_task.o
    0x00000fec   0x00000fec   0x0000004c   Code   RO         1225    i.UIP_ClearEvent    uip_kernel_event.o
    0x00001038   0x00001038   0x000000a4   Code   RO         1324    i.UIP_GetResource   uip_kernel_resource.o
    0x000010dc   0x000010dc   0x000000b0   Code   RO         1273    i.UIP_ReceiveMessage  uip_kernel_message.o
    0x0000118c   0x0000118c   0x00000100   Code   RO         1325    i.UIP_ReleaseResource  uip_kernel_resource.o
    0x0000128c   0x0000128c   0x000000dc   Code   RO         1275    i.UIP_SendMessage   uip_kernel_message.o
    0x00001368   0x00001368   0x000000fc   Code   RO         1227    i.UIP_SetEvent      uip_kernel_event.o
    0x00001464   0x00001464   0x000000f8   Code   RO         1396    i.UIP_TerminateTask  uip_kernel_task.o
    0x0000155c   0x0000155c   0x00000084   Code   RO         1228    i.UIP_WaitEvent     uip_kernel_event.o
    0x000015e0   0x000015e0   0x00000014   Code   RO          903    i.USBD_IRQHandler   chip_uip_interrupt.o
    0x000015f4   0x000015f4   0x00000014   Code   RO          904    i.WDT_IRQHandler    chip_uip_interrupt.o
    0x00001608   0x00001608   0x00000020   Code   RO         1631    i.__0printf$5       mc_p.l(printf5.o)
    0x00001628   0x00001628   0x00000028   Code   RO         1633    i.__0sprintf$5      mc_p.l(printf5.o)
    0x00001650   0x00001650   0x00000008   Code   RO         1779    i.__aeabi_errno_addr  mc_p.l(errno.o)
    0x00001658   0x00001658   0x0000000e   Code   RO         1841    i.__scatterload_copy  mc_p.l(handlers.o)
    0x00001666   0x00001666   0x00000002   Code   RO         1842    i.__scatterload_null  mc_p.l(handlers.o)
    0x00001668   0x00001668   0x0000000e   Code   RO         1843    i.__scatterload_zeroinit  mc_p.l(handlers.o)
    0x00001676   0x00001676   0x00000002   PAD
    0x00001678   0x00001678   0x000002dc   Code   RO         1638    i._printf_core      mc_p.l(printf5.o)
    0x00001954   0x00001954   0x0000000a   Code   RO         1640    i._sputc            mc_p.l(printf5.o)
    0x0000195e   0x0000195e   0x0000000c   Code   RO          408    i.fputc             retarget.o
    0x0000196a   0x0000196a   0x00000002   PAD
    0x0000196c   0x0000196c   0x0000001c   Code   RO          185    i.main              demo.o
    0x00001988   0x00001988   0x00000028   Code   RO          345    i.pre_main_init     init.o
    0x000019b0   0x000019b0   0x000000a8   Code   RO          410    i.stackDump         retarget.o
    0x00001a58   0x00001a58   0x00000024   Code   RO         1139    i.uipAlarmInitialize  uip_kernel_common.o
    0x00001a7c   0x00001a7c   0x00000060   Code   RO          186    i.uipAppInitialize  demo.o
    0x00001adc   0x00001adc   0x00000040   Code   RO         1342    i.uipClearPrioGrpAndArrayBit  uip_kernel_scheduler.o
    0x00001b1c   0x00001b1c   0x00000048   Code   RO         1343    i.uipGetNextPriority  uip_kernel_scheduler.o
    0x00001b64   0x00001b64   0x0000006c   Code   RO         1344    i.uipGetNextTask    uip_kernel_scheduler.o
    0x00001bd0   0x00001bd0   0x00000018   Code   RO          905    i.uipInterruptHandlingCallback  chip_uip_interrupt.o
    0x00001be8   0x00001be8   0x000000ac   Code   RO         1258    i.uipInterruptServiceEngine  uip_kernel_isr_engine.o
    0x00001c94   0x00001c94   0x000000c0   Code   RO         1140    i.uipKernelInitialize  uip_kernel_common.o
    0x00001d54   0x00001d54   0x00000034   Code   RO         1142    i.uipMsgInitialize  uip_kernel_common.o
    0x00001d88   0x00001d88   0x00000028   Code   RO         1345    i.uipPreContexSwitch  uip_kernel_scheduler.o
    0x00001db0   0x00001db0   0x00000048   Code   RO         1144    i.uipResInitialize  uip_kernel_common.o
    0x00001df8   0x00001df8   0x00000028   Code   RO         1346    i.uipResetPrioGrpAndArrayBit  uip_kernel_scheduler.o
    0x00001e20   0x00001e20   0x000000dc   Code   RO         1146    i.uipTaskInitialize  uip_kernel_common.o
    0x00001efc   0x00001efc   0x00000048   Code   RO         1147    i.uipTaskStackInit  uip_kernel_common.o
    0x00001f44   0x00001f44   0x00000038   Data   RO          510    .constdata          clk.o
    0x00001f7c   0x00001f7c   0x00000030   Data   RO          724    .constdata          uart.o
    0x00001fac   0x00001fac   0x00000081   Data   RO         1804    .constdata          mc_p.l(ctype_o.o)
    0x0000202d   0x0000202d   0x00000003   PAD
    0x00002030   0x00002030   0x00000004   Data   RO         1805    .constdata          mc_p.l(ctype_o.o)
    0x00002034   0x00002034   0x00000020   Data   RO         1839    Region$$Table       anon$$obj.o


    Execution Region ER_RW (Exec base: 0x20000000, Load base: 0x00002054, Size: 0x0000036c, Max: 0xffffffff, ABSOLUTE)

    Exec Addr    Load Addr    Size         Type   Attr      Idx    E Section Name        Object

    0x20000000   0x00002054   0x0000002c   Data   RW            5    .data               system_nuc200series.o
    0x2000002c   0x00002080   0x00000018   Data   RW          125    .data               app_cfg.o
    0x20000044   0x00002098   0x00000018   Data   RW          126    .data               app_cfg.o
    0x2000005c   0x000020b0   0x00000030   Data   RW          127    .data               app_cfg.o
    0x2000008c   0x000020e0   0x00000001   Data   RW          128    .data               app_cfg.o
    0x2000008d   0x000020e1   0x00000003   PAD
    0x20000090   0x000020e4   0x00000014   Data   RW          129    .data               app_cfg.o
    0x200000a4   0x000020f8   0x00000001   Data   RW          130    .data               app_cfg.o
    0x200000a5   0x000020f9   0x00000003   PAD
    0x200000a8   0x000020fc   0x00000024   Data   RW          131    .data               app_cfg.o
    0x200000cc   0x00002120   0x00000001   Data   RW          132    .data               app_cfg.o
    0x200000cd   0x00002121   0x00000003   PAD
    0x200000d0   0x00002124   0x00000120   Data   RW          133    .data               app_cfg.o
    0x200001f0   0x00002244   0x00000001   Data   RW          134    .data               app_cfg.o
    0x200001f1   0x00002245   0x00000004   Data   RW          135    .data               app_cfg.o
    0x200001f5   0x00002249   0x00000003   PAD
    0x200001f8   0x0000224c   0x00000020   Data   RW          157    .data               app_int_cfg.o
    0x20000218   0x0000226c   0x00000001   Data   RW          158    .data               app_int_cfg.o
    0x20000219   0x0000226d   0x00000004   Data   RW          159    .data               app_int_cfg.o
    0x2000021d   0x00002271   0x00000003   PAD
    0x20000220   0x00002274   0x00000004   Data   RW          411    .data               retarget.o
    0x20000224   0x00002278   0x00000020   Data   RW         1149    .data               uip_kernel_common.o
    0x20000244   0x00002298   0x00000001   Data   RW         1151    .data               uip_kernel_common.o
    0x20000245   0x00002299   0x00000003   PAD
    0x20000248   0x0000229c   0x00000110   Data   RW         1347    .data               uip_kernel_scheduler.o
    0x20000358   0x000023ac   0x00000001   Data   RW         1348    .data               uip_kernel_scheduler.o
    0x20000359   0x000023ad   0x00000003   PAD
    0x2000035c   0x000023b0   0x00000004   Data   RW         1349    .data               uip_kernel_scheduler.o
    0x20000360   0x000023b4   0x00000001   Data   RW         1350    .data               uip_kernel_scheduler.o
    0x20000361   0x000023b5   0x00000003   PAD
    0x20000364   0x000023b8   0x00000004   Data   RW         1353    .data               uip_kernel_scheduler.o
    0x20000368   0x000023bc   0x00000004   Data   RW         1782    .data               mc_p.l(errno.o)


    Execution Region ER_ZI (Exec base: 0x2000036c, Load base: 0x000023c0, Size: 0x00000b2c, Max: 0xffffffff, ABSOLUTE)

    Exec Addr    Load Addr    Size         Type   Attr      Idx    E Section Name        Object

    0x2000036c        -       0x00000120   Zero   RW          119    .bss                app_cfg.o
    0x2000048c        -       0x00000120   Zero   RW          120    .bss                app_cfg.o
    0x200005ac        -       0x00000120   Zero   RW          121    .bss                app_cfg.o
    0x200006cc        -       0x00000120   Zero   RW          122    .bss                app_cfg.o
    0x200007ec        -       0x00000120   Zero   RW          123    .bss                app_cfg.o
    0x2000090c        -       0x00000120   Zero   RW          124    .bss                app_cfg.o
    0x20000a2c        -       0x00000068   Zero   RW         1148    .bss                uip_kernel_common.o
    0x20000a94   0x000023c0   0x00000004   PAD
    0x20000a98        -       0x00000400   Zero   RW          112    STACK               startup_nuc200series.o


==============================================================================

Image component sizes


      Code (inc. data)   RO Data    RW Data    ZI Data      Debug   Object Name

       104          6          0          0          0       2584   adc.o
         0          0          0        448       1728      11334   app_cfg.o
         4          0          0         37          0       1635   app_int_cfg.o
       724        206          0          0          0      20643   chip_uip_interrupt.o
       912        122         56          0          0       7046   clk.o
       346         78          0          0          0      95945   demo.o
        66         16          0          0          0       1190   hardware_init.o
       422         56          0          0          0      59109   init.o
       280        132          0          4          0       5474   retarget.o
        76         32        192          0       1024        844   startup_nuc200series.o
        26          0          0          0          0        622   sys.o
       146         26          0         44          0     117867   system_nuc200series.o
       224         34         48          0          0       2400   uart.o
       692        102          0         33        104      14933   uip_kernel_common.o
       460         72          0          0          0       3056   uip_kernel_event.o
        88          4          0          0          0        448   uip_kernel_isr_cm.o
       172         32          0          0          0        828   uip_kernel_isr_engine.o
       396         16          0          0          0       2407   uip_kernel_message.o
       420         84          0          0          0       2188   uip_kernel_resource.o
       324         30          0        282          0      12540   uip_kernel_scheduler.o
       464         84          0          0          0       1987   uip_kernel_task.o

    ----------------------------------------------------------------------
      6354       1132        328        872       2860     365080   Object Totals
         0          0         32          0          0          0   (incl. Generated)
         8          0          0         24          4          0   (incl. Padding)

    ----------------------------------------------------------------------

      Code (inc. data)   RO Data    RW Data    ZI Data      Debug   Library Member Name

        30          0          0          0          0         60   _chval.o
       166          0          0          0          0         84   _strtoul.o
        26          0          0          0          0         72   atoi.o
         8          4        133          0          0         60   ctype_o.o
         0          0          0          0          0          0   entry.o
         0          0          0          0          0          0   entry10a.o
         0          0          0          0          0          0   entry11a.o
         8          4          0          0          0          0   entry2.o
         4          0          0          0          0          0   entry5.o
         0          0          0          0          0          0   entry7b.o
         0          0          0          0          0          0   entry8b.o
         8          4          0          0          0          0   entry9a.o
         8          4          0          4          0         60   errno.o
        30          0          0          0          0          0   handlers.o
        36          8          0          0          0         68   init.o
        32          0          0          0          0         68   llshl.o
        34          0          0          0          0         68   llushr.o
       814         56          0          0          0        312   printf5.o
       112          4          0          0          0         76   strtol.o
        44          0          0          0          0         72   uidiv.o
        96          0          0          0          0         84   uldiv.o

    ----------------------------------------------------------------------
      1458         84        136          4          0       1084   Library Totals
         2          0          3          0          0          0   (incl. Padding)

    ----------------------------------------------------------------------

      Code (inc. data)   RO Data    RW Data    ZI Data      Debug   Library Name

      1456         84        133          4          0       1084   mc_p.l

    ----------------------------------------------------------------------
      1458         84        136          4          0       1084   Library Totals

    ----------------------------------------------------------------------

==============================================================================


      Code (inc. data)   RO Data    RW Data    ZI Data      Debug   

      7812       1216        464        876       2860     361908   Grand Totals
      7812       1216        464        876       2860     361908   ELF Image Totals
      7812       1216        464        876          0          0   ROM Totals

==============================================================================

    Total RO  Size (Code + RO Data)                 8276 (   8.08kB)
    Total RW  Size (RW Data + ZI Data)              3736 (   3.65kB)
    Total ROM Size (Code + RO Data + RW Data)       9152 (   8.94kB)

==============================================================================

